:020000040000FA
:040000004BEF4FF083
:08000800056ED8CF06F0E0CF31
:1000100007F00001E9CF0DF0EACF08F0E1CF09F0D9
:10002000E2CF0AF0D9CF0BF0DACF0CF0F3CF14F017
:10003000F4CF15F0FACF16F0FBCF17F000C00FF099
:1000400001C010F002C011F003C012F004C013F0A0
:100050009DA02EEF00F09EB0BFEF27F00FC000F084
:1000600010C001F011C002F012C003F013C004F080
:100070000E8E0DC0E9FF08C0EAFF09C0E1FF0AC00B
:10008000E2FF0BC0D9FF0CC0DAFF14C0F3FF15C0AC
:10009000F4FF16C0FAFF17C0FBFF055007C0E0FFD2
:1000A00006C0D8FF1000F2CF0EF0F29EF76AC40F20
:1000B000F66E000EF722000EF86E0900F5500EBE27
:1000C000F28E1200005EBCE2613FDD83C29C7E20A6
:1000D000A3FD1F419DC3217FFCA2401E5F01E3BD24
:1000E0003E6082DC237D9FC1421CFEA0E1BF5D0318
:1000F00080DE3C62BEE0025CDF81633D7C22C09E0C
:100100001D43A1FF4618FAA427799BC584DA3866F7
:10011000E5BB5907DB856739BAE406581947A5FBE3
:100120007826C49A653BD987045AB8E6A7F91B45D7
:10013000C6987A24F8A6441A99C7257B3A6486D8CB
:100140005B05E7B98CD2306EEDB3510F4E10F2ACB7
:100150002F7193CD114FADF3702ECC92D38D6F31A3
:10016000B2EC0E50AFF1134DCE90722C6D33D18F97
:100170000C52B0EE326C8ED0530DEFB1F0AE4C128B
:1001800091CF2D73CA947628ABF517490856B4EA77
:100190006937D58B5709EBB536688AD495CB297763
:1001A000F4AA4816E9B7550B88D6346A2B7597C957
:1001B0004A14F6A8742AC896154BA9F7B6E80A544B
:1001C000D7896B35F76AD80FF66E010EF722000E4D
:1001D000F86E0900F5501200000180028080800353
:1001E000808080808080800480808080808080808B
:1001F000808080808080800580808080808080807A
:1002000080808080808080808080808080808080EE
:100210008080808080808006808080808080808058
:1002200080808080808080808080808080808080CE
:1002300080808080808080808080808080808080BE
:1002400080808080808080808080808080808080AE
:100250008080808080808007808080808080808017
:10026000808080808080808080808080808080808E
:10027000808080808080808080808080808080807E
:10028000808080808080808080808080808080806E
:10029000808080808080808080808080808080805E
:1002A000808080808080808080808080808080804E
:1002B000808080808080808080808080808080803E
:1002C000808080808080808080808080808080802E
:1002D0008080808080808008F76AEC0FF66E020EC6
:1002E000F722000EF86E0900F5501200000101021D
:1002F00001020203010202030203030401020203DA
:1003000002030304020303040304040501020203BD
:1003100002030304020303040304040502030304A9
:100320000304040503040405040505060102020391
:100330000203030402030304030404050203030489
:10034000030404050304040504050506020303046D
:100350000304040503040405040505060304040559
:100360000405050604050506050606070102020345
:100370000203030402030304030404050203030449
:10038000030404050304040504050506020303042D
:100390000304040503040405040505060304040519
:1003A0000405050604050506050606070203030401
:1003B00003040405030404050405050603040405F9
:1003C00004050506040505060506060703040405DD
:1003D00004050506040505060506060704050506C9
:1003E000050606070506060706070708F76A000F51
:1003F000F66E040EF722000EF86E0900F55012009A
:100400000002080A2022282A8082888AA0A2A8AA9C
:10041000F2CF0EF0F29E2C0FF66E040EF722000EB5
:10042000F86E0900F5500EBEF28E12000A00BE8270
:100430000B00DD820C00FC820D001B830E003A8352
:100440000F00598310007883110097831200B58341
:100450001300D4831400F383150012841600318432
:100460001700508418006F8419008E841A00AD8420
:100470001B00CC841C00EB841D000A851E0029850E
:100480001F00488520006785210086852200A685FB
:100490002300C5852400E4852500038626002286E6
:1004A0002700428628006186290080862A00A086CF
:1004B0002B00BF862C00DF862D00FE862E001E87B7
:1004C0002F003D8730005D8731007D8732009C879B
:1004D0003300BC873400DC873500FC8736001C887D
:1004E00037003C8838005C8839007C883A009C885A
:1004F0003B00BC883C00DC883D00FD883E001D8937
:100500003F003E8940005E8941007F894200A0890A
:100510004300C0894400E1894500028A4600238ADD
:100520004700458A4800668A4900878A4A00A98AA6
:100530004B00CA8A4C00EC8A4D000E8B4E00308B6B
:100540004F00528B5000748B5100968B5200B88B29
:100550005300DB8B5400FD8B5500208C5600438CE0
:100560005700668C5800898C5900AD8C5A00D08C8D
:100570005B00F48C5C00188D5D003C8D5E00608D2E
:100580005F00848D6000A98D6100CD8D6200F28DC9
:100590006300178E64003C8EF2CF0EF0F29EB40F13
:1005A000F66E050EF722000EF86E0900F5500EBE2D
:1005B000F28E1200C8C8C8C8C8C8C7C7C7C7C6C651
:1005C000C6C5C5C5C4C4C3C3C2C1C1C0BFBFBEBD0B
:1005D000BCBBBBBAB9B8B7B6B5B4B3B2B1AFAEADC8
:1005E000ACABA9A8A7A6A4A3A2A09F9D9C9A9998EA
:1005F00096949391908E8D8B898886858381807E59
:100600007C7A7977757472706E6D6B6967666462F7
:10061000615F5D5B5A58565453514F4E4C4A4847A0
:10062000454342403F3D3B3A3837353432302F2E38
:100630002C2B29282625242221201F1D1C1B1A199A
:1006400017161514131211100F0E0D0D0C0B0A09AD
:100650000908070706050504040303030202020153
:100660000101010000000000000000000000010185
:10067000010102020203030304040505060707083B
:1006800009090A0B0C0D0D0E0F101112131415167B
:1006900017191A1B1C1D1F20212224252628292B4F
:1006A0002C2E2F3032343537383A3B3D3F404243D1
:1006B0004547484A4C4E4F51535456585A5B5D5F1C
:1006C0006162646667696B6D6E7072747577797A52
:1006D0007C7E808183858688898B8D8E9091939492
:1006E0009698999A9C9D9FA0A2A3A4A6A7A8A9ABFF
:1006F000ACADAEAFB1B2B3B4B5B6B7B8B9BABBBBB7
:10070000BCBDBEBFBFC0C1C1C2C3C3C4C4C5C5C5D3
:10071000C6C6C6C7C7C7C7C8C8C8C8C8246A286A63
:100720002EA695EF03F0010E246E2FA89AEF03F08A
:10073000010E241A2FAC9FEF03F0010E286E2FAE8E
:10074000A4EF03F0010E281A2850241A286A2EAEAE
:10075000ACEF03F0010E286ED8902E36D8902F36CD
:10076000282CB4EF03F02F802452D8B4B9EF03F053
:100770002E80246A45AEBFEF03F0010E246E45AA19
:10078000C4EF03F0010E241A45A8C9EF03F0010ECF
:10079000241A45A4CEEF03F0010E241AD890453652
:1007A00024504512CBEF27F045B0DBEF03F0800E6D
:1007B000016E0EEF04F045B2E2EF03F0C00E016EE1
:1007C0000EEF04F045B4E9EF03F0E00E016E0EEF1A
:1007D00004F045B6F0EF03F0F00E016E0EEF04F0FA
:1007E00045B8F7EF03F0F80E016E0EEF04F045BACE
:1007F000FEEF03F0FC0E016E0EEF04F045BC05EFBA
:1008000004F0FE0E016E0EEF04F045BE0CEF04F096
:10081000FF0E016E0EEF04F0FF0E016ECDEF27F01C
:1008200004011553D8B403D000011BEF04F00001FC
:10083000C76A230EC66E0401152D02D004D0000134
:10084000000128EF04F00001300EC66E800EC76E66
:10085000000C949A9488949614C415F410EC04F047
:10086000000CA0C331F0246AA1C320F03152D8B4E7
:100870005FEF04F03150CF5CD8A043EF04F0000EDE
:10088000016EC5EF06F09EA04AEF04F0000E016E67
:10089000C5EF06F0CF50315C2A08D8B054EF04F011
:1008A000FF0E2D6E5DEF04F0CF50315C006ED890DE
:1008B00000342D6E2D502D242D266CEF04F09EA0BB
:1008C0006CEF04F09E9020062052D8A46CEF04F048
:1008D000000E016EC5EF06F09E929EA26DEF04F031
:1008E000CCCF22F022A077EF04F079EF04F00000E3
:1008F000000022A27EEF04F081EF04F0000000006F
:10090000000022A486EF04F08BEF04F0000000004A
:1009100000000000000000006B9A6B986B88A4BA7E
:100920006E50A4BA6E50A4AA93EF04F06E50016EFC
:1009300001C023F02D062D52D8A4A1EF04F036EF0C
:1009400004F0233CA6EF04F0A8EF04F093EF04F0CA
:10095000A4AAA8EF04F06ECF23F02D062D52D8A440
:10096000B4EF04F036EF04F02350F2CFA2F3F29E7E
:10097000E2EC00F00301A2BFF28E016E01C022F092
:1009800022500708D8B003D00001D0EF04F00001D6
:1009900022C029F0080ED8802254246ED7EF04F02C
:1009A00022AED5EF04F036EF04F0A8EF04F0A4AACD
:1009B000D7EF04F06ECF23F02D062D52D8A4E3EF2D
:1009C00004F036EF04F02350FF0AF2CFA3F3F29EB7
:1009D000E2EC00F00301A3BFF28E016E01C022F031
:1009E00022500708D8B003D0000107EF05F000013E
:1009F000225024242A6E120E2A5C0C08D8B003EF71
:100A000005F036EF04F0080E242610EF05F0080E6E
:100A1000242622AE0EEF05F036EF04F0D7EF04F0F7
:100A2000A4AA10EF05F06ECF23F02D062D52D8A406
:100A30001CEF05F036EF04F02350F2CFA2F3F29E44
:100A4000E2EC00F00301A2BFF28E016E01C022F0C1
:100A500022500708D8B003D000013FEF05F0000195
:100A6000225024242B6E2F0E2B5C0208D8B03BEFB3
:100A700005F036EF04F0080E242648EF05F0080EC6
:100A8000242622AE46EF05F036EF04F010EF05F015
:100A9000A4AA48EF05F06ECF23F02D062D52D8A45E
:100AA00054EF05F036EF04F02350FF0AF2CFA3F322
:100AB000F29EE2EC00F00301A3BFF28E016E01C0D2
:100AC00022F022500708D8B003D0000177EF05F0DC
:100AD0000001225024242C6E2A502C5CD10F0208D5
:100AE000D8B075EF05F036EF04F080EF05F0080E92
:100AF000242622AE7EEF05F036EF04F048EF05F035
:100B00002A502A242B242B24A00F286E2C50282472
:100B1000D00F286E030E28262830226E22323F0E78
:100B200022162838246E0F0E24162838206E203204
:100B30002032030E20162D6A28BE2D802450222438
:100B400020242D24006ED8900030286E0C0E285ED4
:100B500029502826070E28162A502B5CD8802A54A4
:100B6000266E2852D8B4E2EF05F09E929E929EA285
:100B7000B7EF05F0CCCF22F022A0C1EF05F0C3EF14
:100B800005F00000000022A2C8EF05F0CBEF05F051
:100B900000000000000022A4D0EF05F0D5EF05F022
:100BA000000000000000000000000000050E006EC4
:100BB000002EFED700D000000000282EDBEF05F04D
:100BC000CC6A9E929E929EA2E3EF05F0CCCF22F0DB
:100BD00022A0EDEF05F0EFEF05F00000000022A2EB
:100BE000F4EF05F0F7EF05F000000000000022A48C
:100BF000FCEF05F001EF06F000000000000000002F
:100C0000000000006B9A6B986B88A4BA6E50A4BA6F
:100C10006E50280E2D6E010E226E2252D8B421EF96
:100C200006F0A4AA11EF06F06E50016E01C022F08A
:100C30002D062D52D8A41FEF06F0C3EF06F00DEFDE
:100C400006F02252D8A435EF06F0A4AA25EF06F04C
:100C50006E50016E01C022F02D062D52D8A433EF44
:100C600006F0C3EF06F021EF06F02250F008D8A4FA
:100C700048EF06F026500408D8B046EF06F0A4AAC4
:100C80003FEF06F06E50016E01C022F052EF06F009
:100C900022B852EF06F0A4AA4BEF06F06E50016E98
:100CA00001C022F0286AA4AA53EF06F06E50016E2C
:100CB00001C022F02D062D52D8A461EF06F0C3EF3B
:100CC00006F0223C69EF06F0D8902836288074EFB1
:100CD00006F02252D8A472EF06F0D8902836289059
:100CE00074EF06F036EF04F03F0E28162850320855
:100CF000D8A47DEF06F09BEF06F0A4AA7DEF06F0E6
:100D00006E50016E01C022F02D062D52D8A48BEF3B
:100D100006F0C3EF06F0A4AA8BEF06F06E50016E4A
:100D200001C022F02D062D52D8A499EF06F0C3EF92
:100D300006F053EF06F09E929EA29CEF06F0CCCFF9
:100D400022F022A0A6EF06F0A8EF06F000000000B7
:100D500022A2ADEF06F0B0EF06F0000000000000A8
:100D600022A4B5EF06F0BAEF06F000000000000084
:100D70000000000000000A0ECF6E220ECE6E010EA3
:100D8000016EC5EF06F036EF04F0000CCF500008FE
:100D9000D8B0CFEF06F0000E016E63EF07F0010E42
:100DA0000301A36F0001A3C331F09E903150FD08F1
:100DB000D8B0DDEF06F0FD0E316E3150CF5CD8A01B
:100DC000DDEF06F0CEA6E2EF06F0CECF22F022A0B5
:100DD000ECEF06F0EEEF06F00000000022A2F3EFC9
:100DE00006F0F6EF06F000000000000022A4FBEF82
:100DF00006F000EF07F00000000000000000000017
:100E00000000CC6A9E929EA203EF07F0CCCF22F0A6
:100E100022A00DEF07F00FEF07F00000000022A264
:100E200014EF07F017EF07F000000000000022A405
:100E30001CEF07F021EF07F00000000000000000A9
:100E400000000000E30E326EC950206E3250C96EB1
:100E5000C7A028EF07F08E0E326EC950206E3250B8
:100E6000C96EC7A031EF07F0380E326EC950206E40
:100E70003250C96EC7A03AEF07F0E30E326EC95088
:100E8000206E3250C96EC7A043EF07F08F0E326E4E
:100E9000C950206E3250C96EC7A04CEF07F0C00E8B
:100EA000326EC950206E3250C96EC7A055EF07F0A0
:100EB000E00E326EC950206E3250C96EC7A05EEF90
:100EC00007F0010E016E000C392CACEF07F0435017
:100ED0002E14432403019F6FA06B9FC3A1F3000155
:100EE00031EC04F00152D8B47AEF07F0010E016E34
:100EF000C3EF07F0CF6ACE6A979A8E9A98988F8838
:100F0000C6EC06F0979A8E8A98988F888C82030197
:100F1000A06B020EA16F000131EC04F00152D8B4B5
:100F200096EF07F0010E016EC3EF07F02EC0A0F39D
:100F3000010E0301A16F000131EC04F00152D8B49D
:100F4000A6EF07F0010E016EC3EF07F0000E016E71
:100F5000C3EF07F0C3EF07F043502E1443240301FF
:100F60009F6FA06B9FC3A1F3000131EC04F001520D
:100F7000D8B4BFEF07F0010E016EC3EF07F0000E0B
:100F8000016EC3EF07F00DEF28F04050F00B006E3C
:100F9000003A0F0E00160050036AF2CFA2F3F29E41
:100FA000F6EC01F00301A2BFF28E016E01C02AF03F
:100FB00040500F0B036AF2CFA1F3F29E0001F6EC52
:100FC00001F00301A1BFF28E016E01C029F0246A75
:100FD0009F53D8B403D000016CEF08F00001979A3A
:100FE0008E9A98988F88CF500A08D8B0FCEF07F0F7
:100FF000000E016E18EF09F00B0E0301A36F000144
:10100000A3C331F09E903150FD08D8B00AEF08F02C
:10101000FD0E316E3150CF5CD8A00AEF08F0CEA69D
:101020000FEF08F0CECF22F022A019EF08F01BEF4F
:1010300008F00000000022A220EF08F023EF08F0E3
:1010400000000000000022A428EF08F02DEF08F0B7
:10105000000000000000000000000000CC6A9E922A
:101060009EA230EF08F0CCCF22F022A03AEF08F099
:101070003CEF08F00000000022A241EF08F044EF2E
:1010800008F000000000000022A449EF08F04EEF35
:1010900008F00000000000000000000000002AC06E
:1010A00032F0C950206E3250C96EC7A055EF08F01B
:1010B00029C032F0C950206E3250C96EC7A05EEF11
:1010C00008F0979A8E8A98988F888C82000E016E0D
:1010D00018EF09F018EF09F0979A8E8A98988F8880
:1010E0008C92CF500A08D8B07AEF08F0000E016E4B
:1010F00018EF09F00B0E0301A36F0001A3C331F039
:101100009E903150FD08D8B088EF08F0FD0E316E8A
:101110003150CF5CD8A088EF08F0CEA68DEF08F054
:10112000CECF22F022A097EF08F099EF08F0000050
:10113000000022A29EEF08F0A1EF08F000000000DE
:10114000000022A4A6EF08F0ABEF08F000000000BA
:101150000000000000000000CC6A9E929EA2AEEF4C
:1011600008F0CCCF22F022A0B8EF08F0BAEF08F0D8
:101170000000000022A2BFEF08F0C2EF08F000005C
:101180000000000022A4C7EF08F0CCEF08F0000038
:10119000000000000000000000006B9A6B986B8854
:1011A000A4BA6E50A4BA6E50286A28500708D8A076
:1011B0000FEF09F0A4AADAEF08F06E50016E01C03B
:1011C00022F02250F2CFA0F3F29E6CEC01F003016A
:1011D000A0BFF28E016E01C02BF00001A4AAEEEFB9
:1011E00008F06E50016E01C022F02250F2CFA0F341
:1011F000F29E6CEC01F00301A0BFF28E016E015073
:101200002B26D89024322B500108D8A003D00001FF
:101210000CEF09F00001248E282AD5EF08F0979AE8
:101220008E8A98988F888C822450016E18EF09F06E
:10123000000C0301F351F503F3CF01F0F4CF00F0FC
:10124000F603F3500026F451F503F3500020026E2C
:101250000001000C979A8E8A98988F888C928B9AAE
:10126000C69A8B9ACF500E08D8B03CEF09F0C68AC8
:10127000000E016E2AEF0AF00F0E0301A36F0001AA
:10128000A3C331F09E903150FD08D8B04AEF09F069
:10129000FD0E316E3150CF5CD8A04AEF09F0CEA6DA
:1012A0004FEF09F0CECF22F022A059EF09F05BEF0B
:1012B00009F00000000022A260EF09F063EF09F0DE
:1012C00000000000000022A468EF09F06DEF09F0B3
:1012D000000000000000000000000000CC6A9E92A8
:1012E0009EA270EF09F0CCCF22F022A07AEF09F095
:1012F0007CEF09F00000000022A281EF09F084EFEA
:1013000009F000000000000022A489EF09F08EEF30
:1013100009F00000000000000000000000006B9ACF
:101320006B986B88A4BA6E50A4BA6E50226A246A75
:1013300003019F37A0379F37A0379F37A0379F37CC
:10134000A0379F37A0379F37A037C00E9F170001E7
:10135000A4AAA8EF09F06E50016E286A28500A0866
:10136000D8A00FEF0AF00301A0BF03D00001C1EF26
:1013700009F00001979A8E9A98988F888B8AC7EF08
:1013800009F0979A8E8A98988F888C928B9A22501F
:10139000F2CFA1F3F29E6CEC01F00301A1BFF28E3B
:1013A000016E0150242624500708D8A003D0000164
:1013B000DEEF09F0000128060FEF0AF0A4AADEEF25
:1013C00009F06E50016E01C022F0A4AAE5EF09F009
:1013D0006E50016E01C022F0A4AAECEF09F06E502D
:1013E000016E01C022F02250F2CFA1F3F29E6CEC0C
:1013F00001F00301A1BFF28E016E01C024F00001D3
:10140000A4AA00EF0AF06E50016E01C022F0D8903D
:1014100003019F37A0370001282AAEEF09F08B9A0D
:10142000C68A979A8E8A98988F888C8228500B0843
:10143000D8A41FEF0AF0010E016E2AEF0AF028501F
:101440000908D8A028EF0AF0020E016E2AEF0AF070
:10145000000E016E000C000CC68A979A8E9A98981E
:101460008F889551CB08D8A448EF0AF09651B80858
:10147000D8A448EF0AF001019653D8A403D0000184
:1014800048EF0AF000010101938500014BEF0AF0DB
:10149000010193950001180E0301A36F0001A3C37E
:1014A00031F09E903150FD08D8B059EF0AF0FD0E92
:1014B000316E3150CF5CD8A059EF0AF0CEA65EEF66
:1014C0000AF0CECF22F022A068EF0AF06AEF0AF00D
:1014D0000000000022A26FEF0AF072EF0AF0000095
:1014E0000000000022A477EF0AF07CEF0AF0000071
:1014F00000000000000000000000CC6A9E929EA246
:101500007FEF0AF0CCCF22F022A089EF0AF08BEF18
:101510000AF00000000022A290EF0AF093EF0AF018
:1015200000000000000022A498EF0AF09DEF0AF0EE
:10153000000000000000000000000000AA0E326E53
:10154000C950206E3250C96ECA0E326EC7A0A6EFC7
:101550000AF0C950206E3250C96E2EA4B4EF0AF0C2
:10156000170E326EB6EF0AF0740E326EC7A0B6EFE9
:101570000AF0C950206E3250C96E32C029F00C0EEC
:101580005124020F326EC7A0C3EF0AF0C950206E7B
:101590003250C96E246A24500708D8A0E2EF0AF03E
:1015A0002A6A29A6D5EF0AF02A2A29ACD9EF0AF02F
:1015B0002A2AD89029362AA0DFEF0AF02980242A87
:1015C000CBEF0AF029509519326EC7A0E5EF0AF06B
:1015D000C950206E3250C96E246A24500708D8A022
:1015E00004EF0BF02A6A29A6F7EF0AF02A2A29ACA1
:1015F000FBEF0AF02A2AD89029362AA001EF0BF037
:101600002980242AEDEF0AF029509619326EC7A0DE
:1016100007EF0BF0C950206E3250C96E246A245077
:101620000708D8A026EF0BF02A6A29A619EF0BF0BD
:101630002A2A29AC1DEF0BF02A2AD89029362AA095
:1016400023EF0BF02980242A0FEF0BF02950AA0A70
:10165000326EC7A029EF0BF0C950206E3250C96E10
:10166000246A24500708D8A048EF0BF02A6A29A65C
:101670003BEF0BF02A2A29AC3FEF0BF02A2AD89037
:1016800029362AA045EF0BF02980242A31EF0BF0F0
:101690002950AA0A326EC7A04BEF0BF0C950206E3A
:1016A0003250C96E246A24500708D8A06AEF0BF0A4
:1016B0002A6A29A65DEF0BF02A2A29AC61EF0BF00C
:1016C0002A2AD89029362AA067EF0BF02980242AED
:1016D00053EF0BF02950AA0A326EC7A06DEF0BF042
:1016E000C950206E3250C96E246A24500708D8A011
:1016F0008CEF0BF02A6A29A67FEF0BF02A2A29AC7F
:1017000083EF0BF02A2AD89029362AA089EF0BF014
:101710002980242A75EF0BF02950AA0A326EC7A03F
:101720008FEF0BF0C950206E3250C96E010193B596
:1017300003D00001A4EF0BF000012BEC0AF0378A74
:10174000010E016E60EF0CF0286A28500B08D8A03B
:10175000D6EF0BF0246A24500708D8A0C2EF0BF094
:101760002A6A29A6B5EF0BF02A2A29ACB9EF0BF0AB
:101770002A2AD89029362AA0BFEF0BF02980242AE4
:10178000ABEF0BF0036A2850210FE96E010E032026
:10179000EA6EEF502918326EC7A0CCEF0BF0C9509B
:1017A000206E3250C96E282AA5EF0BF051C02DF0E3
:1017B000286A2D50285CD8B00AEF0CF0246A245017
:1017C0000708D8A0F6EF0BF02A6A29A6E9EF0BF07C
:1017D0002A2A29ACEDEF0BF02A2AD89029362AA024
:1017E000F3EF0BF02980242ADFEF0BF0036A285077
:1017F000950FE96E000E0320EA6EEF502918326E45
:10180000C7A000EF0CF0C950206E3250C96E282AD4
:10181000D9EF0BF0246A24500708D8A022EF0CF06F
:101820002A6A29A615EF0CF02A2A29AC19EF0CF028
:101830002A2AD89029362AA01FEF0CF02980242AC2
:101840000BEF0CF0295001013B19326E0001C7A0CB
:1018500027EF0CF0C950206E3250C96E246A245014
:101860000708D8A046EF0CF02A6A29A639EF0CF039
:101870002A2A29AC3DEF0CF02A2AD89029362AA032
:1018800043EF0CF02980242A2FEF0CF0295001019E
:101890003C19326E0001C7A04BEF0CF0C950206E0E
:1018A0003250C96E326AC7A053EF0CF0C950206E97
:1018B0003250C96EC7A05AEF0CF0378A010E016E84
:1018C0004BEF29F037AC6AEF0CF0379C3790516A38
:1018D0006DEF0CF037823790516A4DEF29F0206A96
:1018E000A4AA70EF0CF06E50016E01C022F02250DD
:1018F000E709FF08D8A481EF0CF0010E226E82EFF9
:101900000CF0226A22A086EF0CF0208EA4AA86EFAB
:101910000CF06E50016E01C022F02250E709FF0862
:10192000D8A497EF0CF0010E226E98EF0CF0226A0B
:1019300022A09CEF0CF0208CA4AA9CEF0CF06E501F
:10194000016E01C022F02250E709FF08D8A4ADEFD4
:101950000CF0010E226EAEEF0CF0226A22A0B2EF64
:101960000CF0208AA4AAB2EF0CF06E50016E01C0F8
:1019700022F02250E709FF08D8A4C3EF0CF0010EB3
:10198000226EC4EF0CF0226A22A0C8EF0CF020886F
:10199000A4AAC8EF0CF06E50016E01C022F02250D4
:1019A000E709FF08D8A4D9EF0CF0010E226EDAEF98
:1019B0000CF0226A22A0DEEF0CF02086A4AADEEF53
:1019C0000CF06E50016E01C022F02250E709FF08B2
:1019D000D8A4EFEF0CF0010E226EF0EF0CF0226AAB
:1019E00022A0F4EF0CF02084A4AAF4EF0CF06E50C7
:1019F000016E01C022F02250E709FF08D8A405EFCC
:101A00000DF0010E226E06EF0DF0226A22A00AEF01
:101A10000DF02082A4AA0AEF0DF06E50016E01C0F5
:101A200022F02250E709FF08D8A41BEF0DF0010EA9
:101A3000226E1CEF0DF0226A22A020EF0DF0208014
:101A4000000C206AA4AA22EF0DF06E50016E01C0B6
:101A500022F02A6A29A62EEF0DF02A2A29AC32EFAD
:101A60000DF02A2AD89029362AA038EF0DF02980C7
:101A70002250E709FF08D8A442EF0DF0010E226EB4
:101A800043EF0DF0226A2950221A22A049EF0DF0EF
:101A9000208EA4AA49EF0DF06E50016E01C022F015
:101AA0002A6A29A655EF0DF02A2A29AC59EF0DF024
:101AB0002A2AD89029362AA05FEF0DF029802250DB
:101AC000E709FF08D8A469EF0DF0010E226E6AEF56
:101AD0000DF0226A2950221A22A070EF0DF0208CFE
:101AE000A4AA70EF0DF06E50016E01C022F02A6AB8
:101AF00029A67CEF0DF02A2A29AC80EF0DF02A2AC6
:101B0000D89029362AA086EF0DF029802250E709C7
:101B1000FF08D8A490EF0DF0010E226E91EF0DF0AA
:101B2000226A2950221A22A097EF0DF0208AA4AA37
:101B300097EF0DF06E50016E01C022F02A6A29A6BF
:101B4000A3EF0DF02A2A29ACA7EF0DF02A2AD8908E
:101B500029362AA0ADEF0DF029802250E709FF08B1
:101B6000D8A4B7EF0DF0010E226EB8EF0DF0226A87
:101B70002950221A22A0BEEF0DF02088A4AABEEFA1
:101B80000DF06E50016E01C022F02A6A29A6CAEF3C
:101B90000DF02A2A29ACCEEF0DF02A2AD89029364A
:101BA0002AA0D4EF0DF029802250E709FF08D8A41D
:101BB000DEEF0DF0010E226EDFEF0DF0226A2950EC
:101BC000221A22A0E5EF0DF02086A4AAE5EF0DF081
:101BD0006E50016E01C022F02A6A29A6F1EF0DF0C5
:101BE0002A2A29ACF5EF0DF02A2AD89029362AA006
:101BF000FBEF0DF029802250E709FF08D8A405EF7C
:101C00000EF0010E226E06EF0EF0226A2950221A03
:101C100022A00CEF0EF02084A4AA0CEF0EF06E5060
:101C2000016E01C022F02A6A29A618EF0EF02A2AB6
:101C300029AC1CEF0EF02A2AD89029362AA022EFD0
:101C40000EF029802250E709FF08D8A42CEF0EF0EF
:101C5000010E226E2DEF0EF0226A2950221A22A0C8
:101C600033EF0EF02082A4AA33EF0EF06E50016E17
:101C700001C022F02A6A29A63FEF0EF02A2A29ACD9
:101C800043EF0EF02A2AD89029362AA049EF0EF009
:101C900029802250E709FF08D8A453EF0EF0010E67
:101CA000226E54EF0EF0226A2950221A22A05AEF17
:101CB0000EF02080000C286A28500708D8A0D0EF2A
:101CC0000EF0A4AA61EF0EF06E50016E2A6A29A6EA
:101CD0006BEF0EF02A2A29AC6FEF0EF02A2AD8906B
:101CE00029362AA075EF0EF02980D89028340301F8
:101CF000A46BA36F820EA325E96E010EA421EA6EE8
:101D0000EF502B5CD8B403D00001B9EF0EF0000106
:101D1000A4AA88EF0EF06E50016E2A6A29A692EFEF
:101D20000EF02A2A29AC96EF0EF02A2AD8902936EE
:101D30002AA09CEF0EF02980D89028340301A46BD0
:101D4000A36F010EA325016E000EA421036E0150A6
:101D5000820FE96E010E0320EA6EEF502C5CD8B4BE
:101D600003D00001B7EF0EF00001010E246ECDEF9D
:101D70000EF0A4AAB9EF0EF06E50016E2A6A29A6E1
:101D8000C3EF0EF02A2A29ACC7EF0EF02A2AD8900A
:101D900029362AA0CDEF0EF02980282A5CEF0EF01C
:101DA000286A28500F08D8A004EF0FF0A4AAD6EF95
:101DB0000EF06E50016E2A6A29A6E0EF0EF02A2A74
:101DC00029ACE4EF0EF02A2AD89029362AA0EAEFAF
:101DD0000EF029802B50CB08D8A401EF0FF02C5027
:101DE000B808D8A401EF0FF001019653D8A403D08E
:101DF000000101EF0FF0000101019385010E246E37
:101E00000001282AD1EF0EF02AEF20F00301F06B39
:101E1000EF6BF16B00010301F1510B08D8B003D057
:101E2000000148EF0FF00001F0C3F2F3EFC3F0F34D
:101E3000F2C3EFF3036A0301F151EA25E96EEB51B6
:101E40000320EA6EEF50F01BF039006E0F0E001603
:101E50000050F01BF039006EF00E00160050EF1B22
:101E6000F031006E003200321F0E00160050EF1BE2
:101E7000F039006EF00E00160050006ED89000365B
:101E80000050F01B00010301F12B00010BEF0FF0DC
:101E90000301F16B00010301EE51F15DD8A003D005
:101EA000000188EF0FF00001F0C3F2F3EFC3F0F38D
:101EB000F2C3EFF3036A0301F151EC25E96EED5132
:101EC0000320EA6EEF50F01BF039006E0F0E001683
:101ED0000050F01BF039006EF00E00160050EF1BA2
:101EE000F031006E003200321F0E00160050EF1B62
:101EF000F039006EF00E00160050006ED8900036DB
:101F00000050F01B00010301F12B00014BEF0FF01B
:101F10000301F46BEFC3F3F3010EF66FF56B0001F1
:101F200019EC09F002C0F4F301C0F3F30301F0511E
:101F3000F325016E000EF421036E0150016E035073
:101F4000026E0001000C0301EC6BED6B000103015C
:101F5000ED510708D8B003D00001D3EF0FF0000116
:101F60000301ED51EB25036AE925E96EEA510320EF
:101F7000EA6EEFCFEFF3030EED25036A210FE96E52
:101F8000010E0320EA6EEF50EF5DD8B403D00001DC
:101F9000CEEF0FF000010301EC2B00010301ED2B4C
:101FA0000001A7EF0FF00301EC510808D8B403D0EB
:101FB0000001E0EF0FF00001010E016E15EF10F0CF
:101FC0000301EC6BED6B00010301ED510708D8B084
:101FD00003D0000106EF10F000010301ED51EB25E5
:101FE000036AE925E96EEA510320EA6EEF3C02D06C
:101FF00004D00001000101EF10F000010301EC2BFF
:1020000000010301ED2B0001E4EF0FF00301EC519F
:102010000808D8B403D0000113EF10F00001010E3E
:10202000016E15EF10F0000E016E000C8B94000C89
:10203000979C8E9C000C9D90379E37A023EF10F04C
:1020400037903792379C16EC10F018EC10F0979AF6
:102050008E9A98988F98000C1BEC10F0000C2CECCA
:1020600010F0000C0301AE6BD1B0AE2BAE51016E7F
:10207000000136EF1DF0030EF66EF76A300EF86EB3
:102080000800F5CFAEF3F86AD8900301AE33AE5135
:10209000016E00013AEF1DF0D190000C0301AE512A
:1020A0000708D8A003D000015AEF10F00001030187
:1020B000AE6B0001D8900301AE35FE0BAF6F00018F
:1020C0004CEC10F00301B06BF2BEB02BB053D8A4AF
:1020D00003D0000172EF10F00001F29CF29EF2BEFC
:1020E0006EEF10F0030EF66EF76A300EF86EAFC3A7
:1020F000F5FF0C00A68EA68CA684550EA76EAA0E20
:10210000A76EA682000000000000F86AA6940301F2
:10211000B053D8A403D0000191EF10F00001C00E1D
:10212000F212000CD180000CB6C342F08D80200E5C
:10213000286E2852D8B4A4EF10F098908F80989011
:102140008F90280699EF10F08D900301B653D8A414
:1021500003D00001B6EF10F0000198908F809890A6
:102160008F900301B6070001A5EF10F0000CAFC37C
:10217000B6F394EC10F0C1EF10F0AEC3AFF3B7EFCD
:1021800010F0A4EF1DF0AEC33AF0000CAEC343F064
:10219000C0EF1DF00101986B976B9A6B996B9C6B6C
:1021A0009B6B9E6B9D6BA06B9F6BA96B010EA86FC9
:1021B000470EA76FA66BA16BA26BA36B9397A46B43
:1021C000A56B93990001000C000CFF0ED880CF5432
:1021D0000301EE6BED6FEEC3F4F3EDC3F3F3F66BB7
:1021E000330EF56F000119EC09F002C0ECF301C0E9
:1021F000EBF30301EB51016EEC51026E000141EF74
:1022000011F0016A026A006A036A0301F051D8B44E
:1022100003D0000113EF11F0EF51D8A403D0000157
:102220003DEF11F00001100E0301F16F0001D89095
:102230000301ED37EE3700360336F051035CD8B4B6
:1022400003D0000127EF11F0EF51005C0001D8A08E
:1022500033EF11F00301EF51005ED8A00306F051F7
:10226000035ED8800001013602360301F12F02D04F
:1022700004D00001000117EF11F00001000CE5EFA0
:1022800010F002C0EAF301C0E9F3C80E0301E95DF2
:10229000EB6F000EEA59EC6FECC3EEF3EBC3EDF31A
:1022A000F06B320EEF6F000101EC11F00150016E86
:1022B000000C006A016A026A036A0401246B256B40
:1022C000266B276B2351221121112011D8A403D092
:1022D0000001B3EF11F00001200E0401286F00018E
:1022E000D89004011C371D371E371F372437253778
:1022F000263727372351275DD8B403D0000192EF4A
:1023000011F02251265DD8B403D0000192EF11F0F4
:102310002151255DD8B403D0000192EF11F0205176
:10232000245D0001D8A0A6EF11F004012051245F24
:102330002151D8A0213D255F2251D8A0223D265F02
:102340002351D8A0233D275FD880000100360136F5
:10235000023603360401282F02D004D00001000108
:1023600070EF11F00001040EEA6E240EE96E000C0D
:1023700004010B510F5DD8B003D0000146EF12F0FD
:102380000001D8A4E5EF11F004010A510E5DD8B0A8
:1023900003D0000146EF12F00001D8A4E5EF11F0E0
:1023A000040109510D5DD8B003D0000146EF12F0D1
:1023B0000001D8A4E5EF11F004010C51085DD8A08C
:1023C00003D0000146EF12F000010BC41FF40AC451
:1023D0001EF409C41DF408C41CF40401236B226B11
:1023E000010E216F080E206F000159EC11F0EFCFA4
:1023F00010F4ECCF11F4ECCF12F4ECCF13F4ED5257
:10240000ED52ED52040108510C5D006E09510D5959
:10241000016E0A510E59026E0B510F59036E005096
:102420001025146F01501121156F02501221166FE3
:1024300003501321176F1753D8B403D0000140EF96
:1024400012F0000104011653D8B403D0000140EF8C
:1024500012F00001040115510008D8A003D00001BA
:1024600044EF12F00001FF0AD8A440EF12F004017B
:1024700014510708D8A003D0000144EF12F0000166
:10248000000E016EA7EF12F0A5EF12F00FC41FF4BB
:102490000EC41EF40DC41DF40CC41CF40401236B03
:1024A000226B010E216F080E206F000159EC11F014
:1024B000EFCF10F4ECCF11F4ECCF12F4ECCF13F417
:1024C000ED52ED52ED5204010C51085D006E0D51BC
:1024D0000959016E0E510A59026E0F510B59036EC4
:1024E00000501025146F01501121156F0250122158
:1024F000166F03501321176F1753D8B403D0000180
:10250000A1EF12F0000104011653D8B403D000016A
:10251000A1EF12F00001040115510008D8A003D06A
:102520000001A5EF12F00001FF0AD8A4A1EF12F0FC
:10253000040114510708D8A003D00001A5EF12F040
:102540000001000E016EA7EF12F0010E016E000CEB
:10255000F29CF29EF2BEA9EF12F0010E0401146F7C
:10256000000129EC04F08C96000CC9CF1FF41DC4A7
:10257000C9FFC7A0B9EF12F0C9CF1EF404011E5164
:10258000016E0001000C8C86C00EF212000CA8EC4B
:1025900012F0570E04011D6F0001B5EC12F004019A
:1025A0001D6B0001B5EC12F001C010F4C3EC12F089
:1025B000040110BF03D00001E5EF12F00001010E8D
:1025C000016EE9EF12F0E9EF12F0000E016EE9EF93
:1025D00012F0000C0401286B296B010E2A6FDA6AD5
:1025E000D96A040E2D6F200E2C6F0001040EEA6EC6
:1025F000240EE96E2DC4E2FF2CC4E1FF2AC42BF4A3
:10260000D890E550EE02F35004012823F45029231A
:102610002B2F02D004D00001000100EF13F028C4DA
:10262000DEFF29C428F4296BD8B0292B2C2BD8B471
:102630002D2B2A2B2A510508D8B403D00001F6EF20
:1026400012F0000152EF13F017C41FF416C41EF469
:1026500015C41DF414C41CF40401236B226B010E79
:10266000216F080E206F000159EC11F001C019F420
:1026700000C018F404011F6B1E6B19C41DF418C4AC
:102680001CF41FC423F41EC422F41DC421F41CC472
:1026900020F4276B266B010E256F080E246F0001B6
:1026A000EAEF12F000500401145D006E015015595C
:1026B000016E02501659026E03501759036E01C085
:1026C0001BF400C01AF4D890183719371BB103D087
:1026D00000016FEF13F00001040118810001040EE6
:1026E000036E190EE96E03C0EAFFEFCF1CF41CC4A1
:1026F0001DF4B5EC12F0040E036E180EE96E03C063
:10270000EAFFEFCF1CF41CC41DF4B5EC12F0040E6C
:10271000036E1A0EE96E03C0EAFFEFCF1CF41CC46F
:102720001DF4B5EC12F0000CA8EC12F0550E0401EB
:102730001D6F0001B5EC12F013C417F412C416F4A7
:1027400011C415F410C414F424EC13F0C3EC12F00B
:1027500008EF14F0C7EC12F00152D8B4AAEF13F04E
:10276000000CA8EC12F0830E04011D6F0001B5EC03
:1027700012F013C417F412C416F411C415F410C4E3
:1027800014F424EC13F0C3EC12F0000CA8EC12F0DB
:10279000530E04011D6F0001B5EC12F013C417F4C1
:1027A00012C416F411C415F410C414F424EC13F07C
:1027B000C3EC12F02EEF14F0A8EC12F0860E040118
:1027C0001D6F0001B5EC12F013C417F412C416F417
:1027D00011C415F410C414F424EC13F0C3EC12F07B
:1027E000000CC7EC12F00152D8A4FBEF13F0000E5E
:1027F000016E48EF14F01F2C24EF14F00FC413F4F3
:102800000EC412F40DC411F40CC410F494EF13F0C0
:10281000AAEC13F01EB018EF14F00BC413F40AC4A2
:1028200012F409C411F408C410F4B1EC13F01E80C2
:10283000020E1F6E0FC41DF00EC41CF00DC41BF061
:102840000CC41AF048EF14F00FC413F40EC412F4C1
:102850000DC411F40CC410F4C6EF13F0AAEC13F07D
:102860001EB03EEF14F00BC413F40AC412F409C4F2
:1028700011F408C410F4DCEC13F01E80010E1F6E7E
:102880000FC41DF00EC41CF00DC41BF00CC41AF0D4
:10289000000C07C41FF406C41EF405C41DF404C4D0
:1028A0001CF40401236B226B010E216F080E206FB4
:1028B000000159EC11F0EFCF00F0ECCF01F0ECCFBC
:1028C00002F0ECCF03F0ED52ED52ED520150026EEA
:1028D0000050016E000C0301FB510008D8A003D08A
:1028E000000185EF14F00001FF0AD8A481EF14F075
:1028F0000301FA510808D8A003D0000185EF14F0B5
:102900000001000E016ED9EF15F0F7C30BF4F6C30A
:102910000AF4F5C309F4F4C308F41DC00FF41CC095
:102920000EF41BC00DF41AC00CF4B8EC11F00152F7
:10293000D8A4B7EF14F0C7EC12F00152D8A4A5EF59
:1029400014F0000E016ED9EF15F01DC00BF41CC081
:102950000AF41BC009F41AC008F4F7C30FF4F6C355
:102960000EF4F5C30DF4F4C30CF4F1EC13F0FAC358
:1029700000F0FBC301F0026A036A00500301F42572
:102980000401046F01500301F5210401056F025099
:102990000301F6210401066F03500301F72104012E
:1029A000076FF7C30BF4F6C30AF4F5C309F4F4C3D5
:1029B00008F407C40FF406C40EF405C40DF404C4EF
:1029C0000CF40001B8EC11F00152D8A4F2EF14F0AD
:1029D000C7EC12F00152D8A4F2EF14F0000E016E11
:1029E000D9EF15F0F7C307F4F6C306F4F5C305F401
:1029F000F4C304F449EC14F002C0FFF301C0FEF389
:102A0000F7C303F4F6C302F4F5C301F4F4C300F40E
:102A1000A8EC12F01F2C15EF15F0840E04011D6FA9
:102A20000001B5EC12F01BEF15F0870E04011D6FCD
:102A30000001B5EC12F00401176B166BFFC315F41F
:102A4000FEC314F4000124EC13F00301FD6BFC6BD6
:102A500000010301FD51FB5DD8B003D00001D5EFAB
:102A600015F00001D8A43EEF15F00301FA51FC5D0A
:102A7000D8A003D00001D5EF15F000010301FE51ED
:102A80000808D8B403D00001A5EF15F00001030138
:102A9000FF2D02D004D000010001A5EF15F00001C8
:102AA0000301FF6BFE6B0001C3EC12F0C7EC12F0E8
:102AB0000152D8A460EF15F0000E016ED9EF15F0A9
:102AC000010E0401005D046F000E0159056F000E38
:102AD0000259066F000E0359076F07C40BF406C4B2
:102AE0000AF405C409F404C408F403C40FF402C4CE
:102AF0000EF401C40DF400C40CF40001F1EC13F069
:102B0000A8EC12F00301FF6BFE6B1F2C02D004D067
:102B10000001000195EF15F00001840E04011D6F06
:102B20000001B5EC12F09BEF15F0870E04011D6F4C
:102B30000001B5EC12F00401176B166BFFC315F41E
:102B4000FEC314F4000124EC13F0F9C303F00301F5
:102B5000F851E96E03C0EAFFEFCF04F404C41DF49A
:102B60000001B5EC12F01E9003C41DF002C41CF06D
:102B700001C41BF000C41AF00301FE2BD8B4FF2BD4
:102B8000010E04010027D8B0012BD8B4022BD8B411
:102B9000032B0301F82BD8B4F92B00010301FC2B04
:102BA000D8B4FD2B000129EF15F0C3EC12F0010E93
:102BB000016EF5EF15F00301F36BF26BEBC3F1F36C
:102BC000EAC3F0F3F3C3F7F3F2C3F6F3F1C3F5F39B
:102BD000F0C3F4F3EDC3F9F3ECC3F8F3EFC3FBF385
:102BE000EEC3FAF300016BEF14F00152D8B4FDEF1D
:102BF00015F0000E016EFFEF15F0010E016E000CD6
:102C000037A007EF16F0010E016E09EF16F0000E67
:102C1000016E000C00EC16F00152D8B41AEF16F059
:102C200037AC17EF16F0379C379019EF16F0379244
:102C30003790516A000C1E9A0101926B816B000162
:102C40000AEC16F0000C0301E953D8B403D00001DC
:102C50002FEF16F00001010E0301E96F000137BEEE
:102C600036EF16F0000E016E5EEF16F037A03DEF66
:102C700016F0000E016E5EEF16F051C022F142C058
:102C800023F152C02CF1010E0301EB6F210EEA6F0C
:102C9000ED6B950EEC6F51C0EEF3000106EC0FF0FA
:102CA00002C054F001C053F054C03BF153C03CF19A
:102CB000E9C350F0522A3780010E016E000C030167
:102CC000E86B0001030EEA6EAE0EE96EE26ADB0EFF
:102CD000E16E3A0E016EE6CFEEFF012E6BEF16F0BD
:102CE000030E0301EA6FAE0EE96FEB6B0001A3EC7C
:102CF0000FF00152D8B411EF18F00301B653D8B455
:102D000003D0000180EF17F000010301B753D8B4DE
:102D100003D0000180EF17F0000101019B53D8B4EC
:102D200003D0000180EF17F0000101019C53D8B4DB
:102D300003D0000180EF17F000010301EA6BBFC36D
:102D4000E9F3E9C39AF10101996B036A0301C051E8
:102D50000101992703509A239A510F08D8B003D044
:102D60000001C4EF16F00001D8A4C0EF16F0010175
:102D70009951A008D8B003D00001C4EF16F00001AB
:102D8000010E0301E86F00010301B82D02D004D049
:102D9000000100014AEF17F000010301B951430897
:102DA000D8B403D000014AEF17F000010301BA5173
:102DB0001408D8B403D000014AEF17F00001030152
:102DC000E853D8A403D000014AEF17F00001CAEC81
:102DD00010F00301EA6BBBC3E9F3E9C398F1010109
:102DE000976B036A0301BC51010197270350982395
:102DF000BDC3A4F1BEC3A5F10001E4EC10F03FECAB
:102E000011F001502508D8B048EF17F0A0C1EBF33E
:102E10009FC1EAF3030E0301ED6FBD0EEC6FEF6B84
:102E2000250EEE6F0001DBEC15F00152D8A448EF3F
:102E300017F0400E01019F27000EA0239E6B010E8C
:102E40009D6F9C6B020E9B6F000100EC16F001520F
:102E5000D8B42DEF17F01BEC16F0A50E956F0E0EE3
:102E6000966F976BC60E986F580E996F020E9A6FF9
:102E70009B6B010E9C6F080E516E1E0E0301E96FD5
:102E8000000123EC16F00152D8B448EF17F0378C4C
:102E90007EEF17F0A50E956F0E0E966F976BC60E10
:102EA000986F580E996F060E9A6FFF0E9B6FFF0E6C
:102EB0009C6F010E9D6F430E9E6F140E9F6FE8C3B3
:102EC000A0F0010E036E990EE96E03C0EAFFEF5009
:102ED000A26F010E036E9A0EE96E03C0EAFFEF5077
:102EE000A16F0E0E516E1E0E0301E96F000123EC5F
:102EF00016F00152D8B47EEF17F0378C11EF18F0AE
:102F0000010E036E9C0EE96E03C0EAFFEF50030151
:102F1000B65DD8B403D0000111EF18F00001010E26
:102F2000036E9B0EE96E03C0EAFFEF500301B75D2D
:102F3000D8B403D0000111EF18F00001E4EC10F058
:102F40003FEC11F001502008D8B0C4EF17F0A0C139
:102F5000EBF39FC1EAF3030E0301ED6FB80EEC6FC4
:102F6000EF6B200EEE6F0001DBEC15F00152D8A4E0
:102F7000C4EF17F0200E01019F27000EA0239CC173
:102F80009EF19BC19DF1000101019E51985DD8B059
:102F900003D0000109EF18F00001D8A4D9EF17F011
:102FA000010197519D5DD8A003D0000109EF18F0F1
:102FB000000100EC16F00152D8B4E1EF17F01BEC61
:102FC00016F0A50E956F0E0E966F976BC60E986F46
:102FD000580E996F020E9A6F010E036E9C0EE96EE9
:102FE00003C0EAFFEF509B6F010E036E9B0EE96E6C
:102FF00003C0EAFFEF509C6F080E516E1E0E0301D6
:10300000E96F000123EC16F00152D8B409EF18F073
:10301000378C020E01019B27000E9C23A26BA16B33
:103020000001010193890001D2EF1DF0A69CA19837
:10303000B1C3A9FFB2C3A8FFA69EA684550EA76E72
:10304000AA0EA76EA682A1A823EF18F0A694A198B5
:1030500050EF18F0A69CB2C3A9FFA69EA680A85068
:10306000016E000C0301AE6B00010301AE510708B5
:10307000D8B003D000016CEF18F00001060E030178
:10308000AE25036AD50FE96E000E0320EA6EEFCF7E
:10309000B0F3AEC3B1F3B0C3B2F3000116EF18F052
:1030A000030E0301AE25036A210F016E010E0322F8
:1030B0000150B06F03C0B1F3AEC3B2F300012AEC0C
:1030C00018F0B1C3EAFFB0C3E9FF01C0EFFF03018D
:1030D000AE2B000135EF18F000EC16F00152D8B419
:1030E00074EF18F01BEC16F0A50E956F0E0E966F90
:1030F000976B6D0E986FC00E996F9A6B060E516E9E
:103100001E0E0301E96F000123EC16F00152D8B442
:103110008BEF18F0378CE1EF1DF0AEC344F00301E4
:10312000AE53D8B403D000019BEF18F0000118ECA7
:1031300010F016EC10F0000C8B84000C979C8E8C19
:10314000000C969E8D9EFA0E0301C66F0001C6C349
:1031500034F0020E345E00000000000000000000A9
:103160000000342EAFEF18F0FA0E0301C66F000115
:10317000C6C334F0020E345E000000000000000000
:1031800000000000342EC0EF18F0968E460E0301AA
:10319000C66F0001C6C334F0020E345E00000000AA
:1031A0000000000000000000342ED2EF18F084AEC2
:1031B000E0EF18F0010E016EE4EF18F0E4EF18F004
:1031C000000E016EE4EF18F001C0C3F3FA0E030124
:1031D000C66F0001C6C334F0020E345E000000006A
:1031E0000000000000000000342EF2EF18F0FA0E8C
:1031F0000301C66F0001C6C334F0020E345E000046
:1032000000000000000000000000342E03EF19F061
:103210000301C32D02D004D00001000117EF19F003
:103220000001000E016E1BEF19F01BEF19F0010EEB
:10323000016E1BEF19F0000C0301C56B00010301C7
:10324000C5510708D8B003D000018AEF19F000017A
:10325000969E8D9EC4C300F00301C551016ED8A493
:1032600003D000013AEF19F00001D8900032012E8E
:1032700035EF19F000A062EF19F00A0E0301C66FD6
:103280000001C6C334F0020E345E000000000000EE
:10329000000000000000342E49EF19F0968E4B0E0E
:1032A0000301C66F0001C6C334F0020E345E000095
:1032B00000000000000000000000342E5BEF19F059
:1032C00085EF19F0500E0301C66F0001C6C334F03C
:1032D000020E345E0000000000000000000000004C
:1032E000342E6EEF19F0968E050E0301C66F0001A5
:1032F000C6C334F0020E345E00000000000000007F
:1033000000000000342E80EF19F00301C52B0001EE
:103310001FEF19F0000C0301C46BC36B0001030124
:10332000C3510708D8B003D00001EAEF19F000013B
:10333000969E8D9E080E0301C66F0001C6C334F031
:10334000020E345E000000000000000000000000DB
:10335000342EA6EF19F0968E040E0301C66F0001FD
:10336000C6C334F0020E345E00000000000000000E
:1033700000000000342EB8EF19F084AED4EF19F03D
:10338000010E006E0301C351016ED8A403D00001E9
:10339000D0EF19F00001D8900036012ECBEF19F0D4
:1033A00000500301C4130001410E0301C66F000168
:1033B000C6C334F0020E345E0000000000000000BE
:1033C00000000000342EE0EF19F00301C32B0001D0
:1033D0008FEF19F00301C451016E0001000C0301CD
:1033E000BB518F08D8A003D00001FCEF19F00001F9
:1033F000020E016E58EF1BF0070E0301BB258F086C
:10340000D8A003D000010AEF1AF00001030E016EEC
:1034100058EF1BF0A1EC18F001C0BEF3CC0E030175
:10342000C46F00011CEC19F00F0E0301C46F000102
:103430001CEC19F0BBC3C4F31CEC19F00301C46B02
:1034400000011CEC19F0BDC303F00301BC51E96E8F
:1034500003C0EAFFEFCFC3F3C3C3C4F300011CEC06
:1034600019F00301BC2BD8B4BD2BBDC303F0BC5174
:10347000E96E03C0EAFFEFCFC3F3C3C3C4F3000197
:103480001CEC19F00301BC2BD8B4BD2BBDC303F059
:10349000BC51E96E03C0EAFFEFCFC3F3C3C3C4F36B
:1034A00000011CEC19F00301BC2BD8B4BD2BBDC32B
:1034B00003F0BC51E96E03C0EAFFEFCFC3F3C3C30F
:1034C000C4F300011CEC19F00301BC2BD8B4BD2BD4
:1034D000BDC303F0BC51E96E03C0EAFFEFCFC3F3F5
:1034E000C3C3C4F300011CEC19F00301BC2BD8B416
:1034F000BD2BBDC303F0BC51E96E03C0EAFFEFCFA3
:10350000C3F3C3C3C4F300011CEC19F00301BC2BCB
:10351000D8B4BD2BBDC303F0BC51E96E03C0EAFFB4
:10352000EFCFC3F3C3C3C4F300011CEC19F00301D4
:10353000BC2BD8B4BD2BBDC303F0BC51E96E03C096
:10354000EAFFEFCFC3F3C3C3C4F300011CEC19F0CF
:103550000301BC2BD8B4BD2B00018BEC19F001C0CA
:10356000C0F38BEC19F001C0C1F3A1EC18F0080E08
:103570000301BC5F000EBD5B0001A1EC18F001C0AF
:10358000BEF3CC0E0301C46F00011CEC19F0550E04
:103590000301C46F00011CEC19F0BBC3C4F31CECA5
:1035A00019F00301C46B00011CEC19F0070E0301B4
:1035B000C46F00011CEC19F00301C46B0D0EC36F46
:1035C00000010301C351C411D8A403D0000136EF98
:1035D0001BF00001FA0E0301C66F0001C6C334F0F0
:1035E000020E345E00000000000000000000000039
:1035F000342EF6EF1AF0FA0E0301C66F0001C6C3AF
:1036000034F0020E345E00000000000000000000F4
:103610000000342E07EF1BF0FA0E0301C66F000105
:10362000C6C334F0020E345E00000000000000004B
:1036300000000000342E18EF1BF0FA0E0301C66FD5
:103640000001C6C334F0020E345E0000000000002A
:10365000000000000000342E29EF1BF00301C351CD
:10366000D8B4C407C3070001E1EF1AF08BEC19F0DE
:1036700001C0C2F30301C251AA08D8A403D00001BB
:103680004CEF1BF000010301C2515508D8B403D020
:10369000000152EF1BF00001010E0301BE6F00019B
:1036A00055EF1BF00301BE6B00010301BE51016E1B
:1036B000000188EF1BF0AEC3B0F3AFC3B1F3020E4D
:1036C0000301BA6F00010301BA510708D8B003D053
:1036D00000017BEF1BF00001036A0301BA51B00F38
:1036E000E96E030E0320EA6EEF6A00010301BA2BB4
:1036F000000163EF1BF0030E0301B96FB00EB86F4A
:10370000BB6BB9C3BDF3B8C3BCF30001EFEF19F055
:103710000150016E89EF1EF0020E386E979A8E9A54
:1037200098988F988C9498968F860301C46B5A0E44
:10373000C36F00010301C351C411D8A403D0000119
:10374000EFEF1BF00001FA0E0301C66F0001C6C3C4
:1037500034F0020E345E00000000000000000000A3
:103760000000342EAFEF1BF0FA0E0301C66F00010C
:10377000C6C334F0020E345E0000000000000000FA
:1037800000000000342EC0EF1BF0FA0E0301C66FDC
:103790000001C6C334F0020E345E000000000000D9
:1037A000000000000000342ED1EF1BF0FA0E0301E0
:1037B000C66F0001C6C334F0020E345E0000000084
:1037C0000000000000000000342EE2EF1BF00301B7
:1037D000C351D8B4C407C30700019AEF1BF042C01D
:1037E000B6F394EC10F09CEC18F00301C46BC80E17
:1037F000C36F00010301C351C411D8A403D0000159
:103800004FEF1CF00001FA0E0301C66F0001C6C3A2
:1038100034F0020E345E00000000000000000000E2
:103820000000342E0FEF1CF0FA0E0301C66F0001EA
:10383000C6C334F0020E345E000000000000000039
:1038400000000000342E20EF1CF0FA0E0301C66FBA
:103850000001C6C334F0020E345E00000000000018
:10386000000000000000342E31EF1CF0FA0E0301BE
:10387000C66F0001C6C334F0020E345E00000000C3
:103880000000000000000000342E42EF1CF0030195
:10389000C351D8B4C407C3070001FAEF1BF016ECFC
:1038A00010F00301C46BC80EC36F00010301C351C4
:1038B000C411D8A403D00001ABEF1CF00001FA0E34
:1038C0000301C66F0001C6C334F0020E345E00006F
:1038D00000000000000000000000342E6BEF1CF020
:1038E000FA0E0301C66F0001C6C334F0020E345E47
:1038F000000000000000000000000000342E7CEFFB
:103900001CF0FA0E0301C66F0001C6C334F0020EAC
:10391000345E000000000000000000000000342EB3
:103920008DEF1CF0FA0E0301C66F0001C6C334F020
:10393000020E345E000000000000000000000000E5
:10394000342E9EEF1CF00301C351D8B4C407C30743
:10395000000156EF1CF09EEC18F0378E9E90FD0E85
:10396000CF6EE80ECE6ECC6A9D80000C8CEC1BF006
:10397000000CD551A508D8A437EF1FF0D6510E087A
:10398000D8A437EF1FF0D851C608D8A487EF1DF090
:10399000D951A808D8A487EF1DF00301A36BA46B2D
:1039A000A56BA66BA76BA86BA96BAA6BAB6BAC6B7B
:1039B00000010301EA6BD50EE96F060EEB6F000103
:1039C000A3EC0FF00152D8B487EF1DF0E3C0A5F3CC
:1039D000E4C0A6F30301A553D8B403D00001FBEF64
:1039E0001CF000010301A653D8B403D00001FBEF83
:1039F0001CF00001FF000301A53D02D004D000012E
:103A0000000110EF1DF000010301A63D02D004D01B
:103A10000001000110EF1DF000012FEC10F0030079
:103A20000301A553D8B403D0000120EF1DF000011D
:103A30000301A653D8A403D0000187EF1DF00001B5
:103A40000301A53D02D004D00001000134EF1DF0B8
:103A500000010301A63D02D004D00001000134EFB3
:103A60001DF0000187EF1DF032EF10F001C0A4F34C
:103A70003BEF10F001C0A3F30301A5513C0DF3503F
:103A8000A625A76FA86BD890A831AC6FA731AB6FF4
:103A9000070EAE6F00014EEC10F092EC10F018EC37
:103AA00010F016EC10F00301AA6BA96B00010301E2
:103AB000AA51AC5DD8B003D0000177EF1DF0000132
:103AC000D8A46CEF1DF00301AB51A95DD8A003D0C1
:103AD000000177EF1DF0000103000000000000006E
:103AE0000301A92BD8B4AA2B000157EF1DF04CEC11
:103AF00010F0A3C3AEF34EEC10F00301A453D8A40E
:103B000003D0000187EF1DF0000192EC10F0D851B6
:103B1000CB08D8A4A4EF1DF0D9510808D8A4A4EF6D
:103B20001DF00301EA6BD50EE96F060EEB6F000185
:103B3000A3EC0FF00152D8B4A4EF1DF0E3C0ADF335
:103B4000ADC3AEF3BDEF10F0D851C608D8A4B2EFA4
:103B50001DF0D951D008D8A4B2EF1DF0DBC0AEF3F0
:103B6000C3EC10F0D8519F08D8A4C0EF1DF0D95174
:103B7000C008D8A4C0EF1DF0DBC0AEF3C6EF10F054
:103B8000D82DC6EF1DF0D92DC6EF1DF0D851C608AF
:103B9000D8A4D2EF1DF0D9515808D8A4D2EF1DF007
:103BA0005FEF16F0D8516D08D8A4E1EF1DF0D951A0
:103BB000C008D8A4E1EF1DF01EA2E1EF1DF032EF26
:103BC00018F0D8517408D8A410EF1EF0D951780815
:103BD000D8A410EF1EF00301EA6BD50EE96F0C0EAE
:103BE000EB6F0001A3EC0FF00152D8B410EF1EF000
:103BF000DBC0AEF38DEC18F0DC53D8B404EF1EF04C
:103C00009CEC18F006EF1EF016EC10F0DD53D8B463
:103C10000EEF1EF09EEC18F010EF1EF018EC10F0F6
:103C2000D8518E08D8A4E5EF1EF0D9511808D8A4B1
:103C3000E5EF1EF00301EA6BD50EE96F0B0EEB6F9B
:103C40000001A3EC0FF00152D8B4E5EF1EF02FEC09
:103C500010F00301C46B140EC36F00010301C351C4
:103C6000C411D8A403D0000183EF1EF00001FA0EA6
:103C70000301C66F0001C6C334F0020E345E0000BB
:103C800000000000000000000000342E43EF1EF092
:103C9000FA0E0301C66F0001C6C334F0020E345E93
:103CA000000000000000000000000000342E54EF6F
:103CB0001EF0FA0E0301C66F0001C6C334F0020EF7
:103CC000345E000000000000000000000000342E00
:103CD00065EF1EF0FA0E0301C66F0001C6C334F093
:103CE000020E345E00000000000000000000000032
:103CF000342E76EF1EF00301C351D8B4C407C307B6
:103D000000012EEF1EF0DBC0AEF3DCC0AFF35BEFC3
:103D10001BF0B6EC1CF00301C46B140EC36F000162
:103D20000301C351C411D8A403D00001E5EF1EF074
:103D30000001FA0E0301C66F0001C6C334F0020E83
:103D4000345E000000000000000000000000342E7F
:103D5000A5EF1EF0FA0E0301C66F0001C6C334F0D2
:103D6000020E345E000000000000000000000000B1
:103D7000342EB6EF1EF0FA0E0301C66F0001C6C363
:103D800034F0020E345E000000000000000000006D
:103D90000000342EC7EF1EF0FA0E0301C66F0001BB
:103DA000C6C334F0020E345E0000000000000000C4
:103DB00000000000342ED8EF1EF00301C351D8B428
:103DC000C407C307000190EF1EF01EBEECEF1EF00B
:103DD000000E016E39EF1FF0D8517308D8A433EFED
:103DE0001FF0D951D808D8A433EF1FF00301EA6BB4
:103DF000D50EE96F060EEB6F0001A3EC0FF0015238
:103E0000D8B433EF1FF000EC16F00152D8B40BEF2A
:103E10001FF01BEC16F0A50E956F0E0E966F976BAC
:103E2000860E986F200E996F080E9A6F30C19BF026
:103E300031C19CF032C19DF033C19EF034C19FF07E
:103E400035C1A0F036C1A1F037C1A2F00E0E516EFF
:103E50001E0E0301E96F000123EC16F00152D8B4E5
:103E600033EF1FF0378C010E016E39EF1FF0000E9B
:103E7000016ED7EF20F01EA642EF1FF0010E016E7B
:103E800044EF1FF0000E016EEEEF20F0378860EF78
:103E900021F0C68A979A8E8A98988F888C82180EFD
:103EA0000301A36F0001A3C331F09E903150FD08C0
:103EB000D8B05DEF1FF0FD0E316E3150CF5CD8A051
:103EC0005DEF1FF0CEA662EF1FF0CECF22F022A052
:103ED0006CEF1FF06EEF1FF00000000022A273EFE6
:103EE0001FF076EF1FF000000000000022A47BEF1F
:103EF0001FF080EF1FF00000000000000000000035
:103F00000000CC6A9E929EA283EF1FF0CCCF22F0DD
:103F100022A08DEF1FF08FEF1FF00000000022A203
:103F200094EF1FF097EF1FF000000000000022A4A4
:103F30009CEF1FF0A1EF1FF0000000000000000048
:103F4000000000006B9A6B986B88A4BA6E50A4BAFC
:103F50006E50640E286E988486A4B6EF1FF0285227
:103F6000D8B4B6EF1FF02806ABEF1FF0988486B4E4
:103F7000C1EF1FF02852D8B4C1EF1FF02806B6EFEA
:103F80001FF0988486A4CCEF1FF02852D8B4CCEF51
:103F90001FF02806C1EF1FF0988486B4D7EF1FF0FA
:103FA0002852D8B4D7EF1FF02806CCEF1FF0080E28
:103FB000006E002EFED76B9A6B986B88A4BA6E5079
:103FC000A4BA6E50A4AAE2EF1FF06E50016E01C0B9
:103FD00022F0206A1E0E286E2852D8B40BEF20F073
:103FE0002050CA08D8B40BEF20F0D8902036A4AAED
:103FF000F7EF1FF06E50016E01C022F02250E7096A
:10400000FF08D8A407EF20F0208008EF20F02090D0
:104010002806ECEF1FF02050CA08D8B414EF20F0A7
:10402000000E016E63EF21F06FEC0CF020C029F060
:104030006FEC0CF020C0A0F321EC0DF020C02BF0B1
:1040400021EC0DF020C02CF0246A010193950001B1
:104050005BEF0EF01EAC2FEF20F0010E246E245209
:10406000D8A437EF20F0000E016E63EF21F0286A2C
:1040700028500B08D8A04BEF20F021EC0DF0036A7C
:1040800028502D0FE96E010E0320EA6E20C0EFFFCD
:10409000282A38EF20F00C0E0301A05DFE0F2D6ED4
:1040A0002D504008D8A003D000015CEF20F00001A3
:1040B000000E016E63EF21F0010193B503D0000102
:1040C0006BEF20F000012BEC0AF0400E2D6E000E7D
:1040D000016E63EF21F0286A2D50285CD8B07FEF85
:1040E00020F021EC0DF0036A2850D50FE96E000E88
:1040F0000320EA6E20C0EFFF282A6CEF20F0286A28
:1041000028500108D8A093EF20F021EC0DF0036AAD
:1041100028503D0FE96E010E0320EA6E20C0EFFF2C
:10412000282A80EF20F0010E0301EB6F2D0EEA6FBD
:10413000ED6BD50EEC6F2DC0EEF3000106EC0FF029
:1041400002C0A2F301C0A1F30301A251036A01015D
:104150003D19286E3E510301A119006EA251036E54
:10416000005028122852D8A403D00001C0EF20F03C
:1041700000010101406B000E016E000163EF21F0B0
:10418000D551A508D8A4D7EF20F0D6510E08D8A451
:10419000D7EF20F0010193A103D00001D7EF20F069
:1041A0000001010E0101406F0001B9EF1CF0D55173
:1041B000A508D8A4E8EF20F0D6510E08D8A4E8EF5F
:1041C00020F0010193B303D0000161EF21F0000161
:1041D000020E0101406F00013BEF1FF00152D8A415
:1041E00061EF21F0286A28500B08D8A016EF21F0C3
:1041F000036A2850150F016E010E032201500301BE
:10420000A36F03C0A4F3036A28502D0FE96E010EBB
:104210000320EA6EEF50A56FA4C3EAFFA3C3E9FF32
:10422000A5C3EFFF0001282AF3EF20F0286A2D50E4
:10423000285CD8B03AEF21F0036A2850550F016E80
:10424000000E032201500301A36F03C0A4F3036A0D
:104250002850D50FE96E000E0320EA6EEF50A56FCF
:10426000A4C3EAFFA3C3E9FFA5C3EFFF0001282A07
:1042700017EF21F0286A28500108D8A05EEF21F03E
:10428000036A2850390F016E010E03220150030109
:10429000A36F03C0A4F3036A28503D0FE96E010E1B
:1042A0000320EA6EEF50A56FA4C3EAFFA3C3E9FFA2
:1042B000A5C3EFFF0001282A3BEF21F046EF1FF0D6
:1042C0001E88010E016E5AEF29F037A86CEF21F01D
:1042D000010E016E6EEF21F0000E016EA3EF21F0D2
:1042E00037AA77EF21F0010E016E79EF21F0000E71
:1042F000016E000C70EC21F00150016E000C445274
:10430000D8A483EF21F04452D8B490EF21F03CA21E
:104310008EEF21F09CEC18F090EF21F016EC10F0ED
:10432000442C9CEF21F0382C9AEF21F09EEC18F0F1
:104330009CEF21F018EC10F044500308D8A4ADEF26
:1043400021F065EF21F00152D8B4ABEF21F09EECE3
:1043500018F0ADEF21F018EC10F044500208D8A48A
:10436000BEEF21F07AEC21F00152D8B4BCEF21F07D
:104370009EEC18F0BEEF21F018EC10F04450060847
:10438000D8A4ECEF21F001014051020A0001D8B499
:10439000D4EF21F0030AD8B4DAEF21F0010AD8B43F
:1043A000E0EF21F0E6EF21F09EEC18F016EC10F0B3
:1043B000ECEF21F09EEC18F016EC10F0ECEF21F091
:1043C00018EC10F09CEC18F0ECEF21F018EC10F069
:1043D00016EC10F0ECEF21F078EF29F000EC16F07D
:1043E0000152D8B402EF22F050065052D8A402EF86
:1043F00022F0379037AC00EF22F0379C01EF22F02B
:104400003792516A8DEF29F000EC16F00152D8B4C2
:1044100010EF22F0010E016E14EF22F014EF22F0E3
:10442000000E016E14EF22F0000CAAEC13F01EB087
:1044300035EF22F01F2C2AEF22F01DC013F41CC010
:1044400012F41BC011F41AC010F4B1EC13F01E806A
:1044500035EF22F01DC013F41CC012F41BC011F480
:104460001AC010F4DCEC13F01E80AAEC13F083EFFA
:1044700025F0C7EC12F00152D8A443EF22F0000E51
:10448000016EA4EF22F0A8EC12F0680E04011D6F7B
:104490000001B5EC12F0D7C317F4D6C316F4D5C398
:1044A00015F4D4C314F424EC13F004011D6B0001C3
:1044B000B5EC12F004011D6B0001B5EC12F0040123
:1044C0001D6B0001B5EC12F004011D6B0001B5EC91
:1044D00012F00301DD6BDC6B00010301DD51DB5DDC
:1044E000D8B003D00001A0EF22F00001D8A482EFE1
:1044F00022F00301DA51DC5DD8A003D00001A0EF67
:1045000022F00001D9C303F00301D851DE6F03C0CC
:10451000DFF304011D6B0001B5EC12F0DFC3EAFF0D
:10452000DEC3E9FF01C0EFFF0301D82BD8B4D92BBC
:1045300000010301DC2BD8B4DD2B00016DEF22F06C
:10454000C3EC12F0010E016E000CC7EC12F0015228
:10455000D8A4AFEF22F0000E016EFDEF24F0C3C32C
:104560000BF4C2C30AF4C1C309F4C0C308F41DC0EC
:104570000FF41CC00EF41BC00DF41AC00CF4B8EC00
:1045800011F00152D8B47DEF23F0C3C307F4C2C3C6
:1045900006F4C1C305F4C0C304F449EC14F002C02E
:1045A000C9F301C0C8F3C7C3CDF3C6C3CCF3A8ECAD
:1045B00012F01F2CF1EF22F0540E04011D6F0001C8
:1045C000B5EC12F0C3C317F4C2C316F4C1C315F49B
:1045D000C0C314F424EC13F004011D6B0001B5EC0E
:1045E00012F01F500208D8A40BEF23F0560E04015E
:1045F0001D6F0001B5EC12F0C3C317F4C2C316F46B
:10460000C1C315F4C0C314F424EC13F004011D6BF2
:104610000001B5EC12F00301C651C711D8A403D0B4
:10462000000148EF23F000010301C8510808D8B485
:1046300003D0000128EF23F000010301C92D02D0AF
:1046400004D00001000128EF23F0000148EF23F01F
:10465000C5C303F00301C451D06F03C0D1F30401FB
:104660001D6B0001B5EC12F0D1C3EAFFD0C3E9FF26
:1046700001C0EFFF0301C42BD8B4C52BC82BD8B49D
:10468000C92BC651D8B4C707C60700010BEF23F0EA
:10469000C3EC12F00301C651C711D8A403D0000126
:1046A00079EF23F000010301C651CC5D006EC751C4
:1046B000CD59036E0050C025D06F0350C121D16F7A
:1046C000000EC221D26F000EC321D36FD3C3D7F324
:1046D000D2C3D6F3D1C3D5F3D0C3D4F3C5C3D9F372
:1046E000C4C3D8F3C7C3DBF3C6C3DAF3000139ECA4
:1046F00022F0010E016EFDEF24F00301C3511D5C99
:10470000D8B003D00001E9EF24F00001D8A4AAEF4B
:1047100023F00301C2511C5CD8B003D00001E9EFC3
:1047200024F00001D8A4AAEF23F00301C1511B5CBF
:10473000D8B003D00001E9EF24F00001D8A4AAEF1B
:1047400023F00301C0511A5CD8B003D00001E9EF97
:1047500024F000010301C651C025D06FC751C1210B
:10476000D16F000EC221D26F000EC321D36F1D5036
:10477000D35DD8B003D00001E9EF24F00001D8A444
:10478000E3EF23F01C500301D25DD8B003D0000149
:10479000E9EF24F00001D8A4E3EF23F01B5003015C
:1047A000D15DD8B003D00001E9EF24F00001D8A416
:1047B000E3EF23F01A500301D05DD8B003D000011D
:1047C000E9EF24F00001C7C3CDF3C6C3CCF3030166
:1047D000C0511A5CD06FC1511B58D16FC2511C58C7
:1047E000D26FC3511D58D36F1DC007F41CC006F40F
:1047F0001BC005F41AC004F4000149EC14F002C017
:1048000003F001500301D05DCE6F0350D159CF6F3B
:10481000C96BC86BC3C3D7F3C2C3D6F3C1C3D5F347
:10482000C0C3D4F3C5C3D9F3C4C3D8F3CFC3DBF338
:10483000CEC3DAF3000139EC22F00301CE51C65F9A
:10484000CF51C75BCE51C427CF51C5230001A8EC7F
:1048500012F01F2C4FEF24F0540E04011D6F0001C5
:10486000B5EC12F00301CE51C025D06FCF51C1215C
:10487000D16F000EC221D26F000EC321D36FD3C3FC
:1048800017F4D2C316F4D1C315F4D0C314F4000145
:1048900024EC13F004011D6B0001B5EC12F01F5065
:1048A0000208D8A477EF24F0560E04011D6F000112
:1048B000B5EC12F00301CE51C025D06FCF51C1210C
:1048C000D16F000EC221D26F000EC321D36FD3C3AC
:1048D00017F4D2C316F4D1C315F4D0C314F40001F5
:1048E00024EC13F004011D6B0001B5EC12F0030180
:1048F000C651C711D8A403D00001B4EF24F00001C1
:104900000301C8510808D8B403D0000194EF24F083
:1049100000010301C92D02D004D00001000194EF71
:1049200024F00001B4EF24F0C5C303F00301C45127
:10493000D06F03C0D1F304011D6B0001B5EC12F080
:10494000D1C3EAFFD0C3E9FF01C0EFFF0301C42BCD
:10495000D8B4C52BC82BD8B4C92BC651D8B4C707F7
:10496000C607000177EF24F0C3EC12F00301C65133
:10497000C711D8A403D00001E5EF24F00001030122
:10498000C651CC5D006EC751CD59036E0050C02595
:10499000D06F0350C121D16F000EC221D26F000E23
:1049A000C321D36FD3C3D7F3D2C3D6F3D1C3D5F3C7
:1049B000D0C3D4F3C5C3D9F3C4C3D8F3C7C3DBF39F
:1049C000C6C3DAF3000139EC22F0010E016EFDEFEF
:1049D00024F0C3C3D7F3C2C3D6F3C1C3D5F3C0C356
:1049E000D4F3C5C3D9F3C4C3D8F3C7C3DBF3C6C379
:1049F000DAF339EC22F0010E016E19EF25F0030114
:104A0000BF6BBE6BB7C3BDF3B6C3BCF3BFC3C3F3C9
:104A1000BEC3C2F3BDC3C1F3BCC3C0F3B9C3C5F3C6
:104A2000B8C3C4F3BBC3C7F3BAC3C6F30001A5EF51
:104A300022F00152D8B421EF25F0000E016E23EFD1
:104A400025F0010E016E000CB7C301F0B6C300F0F3
:104A50000066012A0900F5CFEEFF002E2AEF25F0AF
:104A6000012E2AEF25F0F86A05EF26F0B9C303F00E
:104A70000301B851E96E03C0EAFFEF50BC6FBBC33E
:104A800003F0BA51E96E03C0EAFFEF50BD6FBDC33A
:104A9000BEF3BCC3BDF3BEC3BCF3B751BD1BBD3930
:104AA000006E0F0E00160050BD1BBD39006EF00EDB
:104AB00000160050BC1BBD31006E003200321F0ECC
:104AC00000160050BC1BBD39006EF00E00160050E1
:104AD000006ED89000360050BD1BB9C303F0B8512A
:104AE000E96E03C0EAFFBCC3EFFFBBC303F0BA51DA
:104AF000E96E03C0EAFFBDC3EFFF0001000C2FEC1D
:104B000010F015EF22F09CEC18F09EEC18F0030169
:104B1000A06BA16B0101A06B400E9F6FA96B010EF2
:104B2000A86F470EA76FA66B0001E4EC10F003011D
:104B3000B76BB66B030EB96FA60EB86FBB6B100EDA
:104B4000BA6F0001FFEC24F00301B76BA8C3B6F302
:104B5000B6C3A5F3A46B036AA951A4270350A523E8
:104B6000A36BA26B00010301A351A55DD8B003D0D4
:104B700000013EEF26F00001D8A4C8EF25F00301A4
:104B8000A451A25DD8A003D000013EEF26F00001A1
:104B90000301A3511108D8B003D00001F4EF25F0B0
:104BA0000001D8A4DDEF25F00301A2512F08D8B0F1
:104BB00003D00001F4EF25F00001A0C1B7F39FC1BD
:104BC000B6F3030E0301B96FA60EB86FBB6B100EE0
:104BD000BA6F0001FFEC24F0100E01019F27000EB8
:104BE000A02300010FEF26F0A8C1F8FFA7C1F7FF2F
:104BF000A6C1F6FF030EEA6EA60EE96E0301B76BBF
:104C0000100EB66F000124EF25F0100E0101A6274B
:104C1000000EA723000EA823000EA9230001030104
:104C20009F6B000103019F510F08D8B003D0000112
:104C300037EF26F00001036A03019F51A60FE96ECA
:104C4000030E0320EA6EEFCFB6F3B6C3B7F3030E3D
:104C5000B96FA00EB86F030EBB6FA10EBA6F000143
:104C600036EC25F003019F2B000112EF26F0030123
:104C7000A22BD8B4A32B0001B3EF25F0A4C1B7F346
:104C8000030E0301B96FA00EB86F030EBB6FA10E28
:104C9000BA6F000136EC25F0A5C1B7F3030E03018E
:104CA000B96FA00EB86F030EBB6FA10EBA6F0001F3
:104CB00036EC25F0B6EC1CF00301A053D8B403D0B9
:104CC000000172EF26F000010301A153D8B403D014
:104CD000000172EF26F00001010E016E76EF26F062
:104CE00076EF26F0000E016E76EF26F0CCEF26F080
:104CF0002FEC10F0F29CF29EF2BE7BEF26F0010E3C
:104D0000FB6EF90EFA6EB20EF96E00EF98F000EF3E
:104D1000F8F000EFF8F000EF78F01AEF27F001015B
:104D200093A903D0000190EF27F0000101019851F1
:104D30009C5DD8B003D0000120EF27F00001D8A47B
:104D4000ABEF26F001019B51975DD8A003D0000185
:104D500020EF27F0000104EC22F00152D8A420EF4C
:104D600027F00101A3510E08D8B003D0000111EFC4
:104D700027F0000100EC16F00152D8B4C2EF26F083
:104D80001BEC16F00101A353D8B403D00001D7EFF8
:104D900026F000017FEF25F001B0D4EF26F00101ED
:104DA00093970001D7EF26F0010193870001A50E2C
:104DB000956F0E0E966F976BC60E986F580E996F83
:104DC000030E9A6F010193B703D00001FBEF26F0A9
:104DD0000001010E036E9E0EE96E03C0EAFFEF5064
:104DE0009B6F010E036E9D0EE96E03C0EAFFEF504C
:104DF0009C6FFFEF26F0CC0E9B6FCC0E9C6F080EC5
:104E0000516E1E0E0301E96F000123EC16F00152F2
:104E1000D8B40CEF27F0378C0101A32B00011EEF53
:104E200027F0010193B703D000011CEF27F0000128
:104E300078EF26F01EEF27F0CAEC10F08BEF27F08A
:104E400001019B53D8B403D0000130EF27F00001DB
:104E500001019C53D8A403D000018BEF27F000017F
:104E60000101A2516408D8A003D000013DEF27F052
:104E70000001CAEC10F08BEF27F00101A1510508E9
:104E8000D8A003D0000182EF27F0000104EC22F04B
:104E90000152D8A482EF27F000EC16F00152D8B4EA
:104EA00054EF27F01BEC16F0A50E956F0E0E966FC3
:104EB000976BC60E986F580E996F020E9A6F010E7F
:104EC000036E9E0EE96E03C0EAFFEF509B6F010E6A
:104ED000036E9D0EE96E03C0EAFFEF509C6F080E53
:104EE000516E1E0E0301E96F000123EC16F0015212
:104EF000D8B47CEF27F0378C0101A16BA22B000105
:104F00008BEF27F004EC22F00152D8A48BEF27F0AE
:104F10000101A12B000101019399000192EF27F0FB
:104F20000101939900018FEF29F0B250016E000C3E
:104F300095EC27F00150016E000CB350016E000C8F
:104F40009DEC27F00150016E000C98EC27F0A0ECCE
:104F500027F001C09FF303012A519F5DD8A003D021
:104F60000001B7EF27F000010301292B00019FC3C7
:104F70002AF3BDEF27F0A5EF27F094EF29F0C1EF5A
:104F800027F0010E366E379A1E98030E0101406F0E
:104F900000018EEF03F0D4EF03F001C040F09E90CB
:104FA0000401146B000129EC04F0C68A040E6F6E34
:104FB0006C946C886C8E6C9C6B8E6B9A6B9C6B98F3
:104FC0006C9A6B8E979A8E8A98988F888C823950BB
:104FD0000A08D8A4EEEF27F0AEEF28F038506308A7
:104FE000D8A4F5EF27F01FEF28F038500208D8A416
:104FF000FCEF27F003EF28F0382C01EF28F0AEEF9C
:1050000028F098EF29F0060E366E9D90979A8E8ABA
:1050100098988F888C8264EF07F00152D8B418EF0B
:1050200028F0010E386E3B6AFEEF28F01DEF28F0E5
:10503000CF6A960ECE6E60EF29F060EF29F0630E16
:10504000366E9D90979A8E8A98988F888C820301ED
:10505000A06B010EA16F000131EC04F001C022F041
:105060002252D8B4ACEF28F0979A8E9A98988F88ED
:10507000CF500E08D8B03FEF28F060EF29F00F0EA8
:105080000301A36F0001A3C331F09E903150FD08CE
:10509000D8B04DEF28F0FD0E316E3150CF5CD8A066
:1050A0004DEF28F0CEA652EF28F0CECF22F022A06E
:1050B0005CEF28F05EEF28F00000000022A263EF12
:1050C00028F066EF28F000000000000022A46BEF3B
:1050D00028F070EF28F00000000000000000000041
:1050E0000000CC6A9E929EA273EF28F0CCCF22F0F3
:1050F00022A07DEF28F07FEF28F00000000022A220
:1051000084EF28F087EF28F000000000000022A4C0
:105110008CEF28F091EF28F0000000000000000064
:1051200000000000AA0E326EC950206E3250C96EC7
:10513000C7A098EF28F026C032F0C950206E325038
:10514000C96EC7A0A1EF28F0326AC950206E325054
:10515000C96EC7A0A9EF28F060EF29F0020E366EE5
:105160003A502E5CD8B0C2EF28F03B500408D8A0CB
:10517000C2EF28F0979A8E9A98988F88C6EC06F01E
:10518000D9EF28F0979A8E8A98988F888C820A0E89
:105190000301A06F010EA16F000131EC04F001C00A
:1051A00022F02252D8B4D8EF28F03B6AD9EF28F089
:1051B0003B2A39500A08D8A4E0EF28F060EF29F024
:1051C000E2EF28F0030E366E1E942EAAF7EF28F0B9
:1051D000010E03019F6F0001C5EC07F001C040F014
:1051E0003B52D8A4F5EF28F01E84FCEF28F0030111
:1051F0009F6B0001C5EC07F0FEEF28F0040E366E41
:105200000301F46B2FC0F3F3010EF66FF56B000191
:1052100019EC09F002C03FF001C03EF02E503E26CE
:10522000000E3F22CF500E08D8B019EF29F060EFE2
:1052300029F037A032EF29F03FC0A0F33EC09FF322
:105240002AEC09F001C020F0202C29EF29F040EFD2
:1052500029F020500208D8A430EF29F04FEF29F0B0
:105260003EEF29F00301A06B9F6B00012AEC09F0CF
:105270000152D8B43EEF29F04FEF29F060EF29F04A
:10528000050E366ECF501708D8B049EF29F060EF01
:1052900029F02CEF0AF062EF0CF060EF29F0080E15
:1052A000366ECF501708D8B058EF29F060EF29F0CC
:1052B00049EF1FF00152D8A45EEF29F060EF29F00A
:1052C000140E366E979A8E8A98988F888C82326ADE
:1052D000C950206E3250C96E6B9E8B9AC69A979AAF
:1052E0008E9A98988F983C2AD8B43D2A7FEF21F067
:1052F000382C82EF29F03B500708D8B082EF29F014
:10530000020E386E9E9037AE89EF29F09D808BEFAC
:1053100029F01BEC10F0EEEF21F08FEF26F01EB21B
:1053200094EF29F0BBEF27F0000E016EA0EF29F0FB
:105330000A0E366E9CEC18F016EC10F060EF29F0B7
:105340009E902EEF00F0C26A0D0EC16E060EC06E6A
:1053500033EF2BF003013051000A0001D8B4BBEF4A
:1053600029F0010AD8B4D3EF29F0030AD8B4EBEF3F
:1053700029F009EF2AF0EF0E926E806AFF0E936E0D
:10538000816AD30E946E826A730E956E0C0E836ED4
:10539000CC0E966E846A0B0E976E856AE40E986E3C
:1053A000866A09EF2AF0D30E926E806AFF0E936E22
:1053B000816AC30E946E826A020E956E840E836EAD
:1053C0000C0E966E846A1A0E976E856AE40E986EBD
:1053D000866A09EF2AF0FF0E926EFF0E806EFF0EB6
:1053E000936EFF0E816EFF0E946EFF0E826EFF0EA7
:1053F000956EFF0E836EFF0E966EFF0E846EFF0E8F
:10540000976EFF0E856EFF0E986EFF0E866E09EF8B
:105410002AF0010E016E38EF2BF003013251F90F23
:10542000D8A003D0000135EF2AF0070F000136EFB6
:105430002AF00F0EC16E35EF2AF00E0EC16E35EF59
:105440002AF00D0EC16E35EF2AF00C0EC16E35EF4D
:105450002AF00B0EC16E35EF2AF00A0EC16E35EF41
:105460002AF0090EC16E35EF2AF0000CF2CF0EF0D3
:10547000F29EE824970FF66E540EF76ED8B0F72A16
:10548000000EF86EFB6E0A00F550FA6E0800F5503B
:105490000EBEF28EF96E32543A5442544A5452546B
:1054A0005A546254C150F00B0301316F3051FB0F5D
:1054B000D8A003D0000189EF2AF0050F00018BEF7F
:1054C0002AF0020E0301326F00010DEC2AF089EF81
:1054D0002AF0030E0301326F00010DEC2AF089EF70
:1054E0002AF0040E0301326F00010DEC2AF089EF5F
:1054F0002AF0050E0301326F00010DEC2AF089EF4E
:105500002AF0060E0301326F00010DEC2AF089EF3C
:105510002AF03DEF2BF0F2CF0EF0F29EE824410F7F
:10552000F66E550EF76ED8B0F72A000EF86EFB6EC9
:105530000A00F550FA6E0800F5500EBEF28EF96EB4
:10554000C254D254E254F25402558C8EABEF2AF07E
:10555000959EA5EF2AF09596C3EC12F00301C46B5B
:10556000640EC36F00010301C351C411D8A403D05A
:10557000000108EF2BF00001FA0E0301C66F0001D5
:10558000C6C334F0020E345E0000000000000000CC
:1055900000000000342EC8EF2AF0FA0E0301C66F97
:1055A0000001C6C334F0020E345E000000000000AB
:1055B000000000000000342ED9EF2AF0FA0E03019B
:1055C000C66F0001C6C334F0020E345E0000000056
:1055D0000000000000000000342EEAEF2AF0FA0E6E
:1055E0000301C66F0001C6C334F0020E345E000032
:1055F00000000000000000000000342EFBEF2AF045
:105600000301C351D8B4C407C3070001B3EF2AF0A4
:10561000FF0E1D6EFF0E1C6EFF0E1B6EFF0E1A6E30
:10562000010E1F6E1E803FEF2BF08D96000C96969C
:1056300015EC2BF0140E356E000E016E41EF2BF0C1
:105640008D8C000C968E969C20EC2BF043EF2BF06B
:10565000938095908C8045EF2BF09380958047EF59
:105660002BF0A3EF29F00301306B0001AAEF29F022
:105670000301306B000152EF2AF0A8EF2AF017EF78
:105680002BF022EF2BF028EF2BF02DEF2BF01E92BA
:1056900097869692978E8D9260EF4FF00301306B54
:1056A0000001030130513208D8B003D0000175EF7A
:1056B0002BF00001036A03013051AC0FE96E010EBB
:1056C0000320EA6EF2CF33F3F29EAA6A30C3A9FF39
:1056D000A69CA69EA680A85033BFF28EEF6E000156
:1056E0000301302B000151EF2BF0000E016E62EF31
:1056F0004FF08E0E006E92C301F091C302F0036A68
:105700000152D8A490EF2BF002C001F0026A080EFB
:10571000005E0152D8A490EF2BF0006A9AEF2BF0B4
:10572000D89001BE99EF2BF002360136000690EFBB
:105730002BF0019E000C03019151D8A403D000016D
:10574000F9EF2CF09D6F9551D8A403D00001F9EF2B
:105750002CF09D5FD8A003D00001B2EF2BF0000128
:10576000BDEF2BF07F0E03019D27D8A003D00001D1
:10577000F9EF2CF00001CBEF2BF0810E03019D5FC0
:10578000D8B003D00001F9EF2CF0D8A403D0000169
:10579000F9EF2CF000019DC300F0016A026A036A70
:1057A00003019C6B92C39BF39B8F93C39AF394C3A7
:1057B00099F3190E9D6F000103019851995FD8A0CC
:1057C00003D00001FFEF2BF0010E9A5FD8A003D0A9
:1057D0000001FFEF2BF09B5FD8A003D00001FFEF8B
:1057E0002BF09C5FD8A003D00001FFEF2BF09C2B87
:1057F0009B2B9A2B98519927000159EF2CF003010C
:1058000097519A5FD8A003D0000133EF2CF0010E1E
:105810009B5FD8A003D0000133EF2CF09C5FD8A091
:1058200003D0000133EF2CF0000103019C2B9B2BD4
:1058300097519A270001030198519927D8B003D0B6
:10584000000159EF2CF09A2BD8B403D0000159EF86
:105850002CF09B2BD8B403D0000159EF2CF09C2BDB
:10586000000159EF2CF00301965180099B5FD8A0ED
:1058700003D0000158EF2CF0010E9C5FD8A003D09C
:10588000000158EF2CF09C2B965180099B279751D3
:105890009A27D8B003D000011BEF2CF09B2BD8B473
:1058A00003D000011BEF2CF09C2B00011BEF2CF010
:1058B000038003019D2F02D004D00001000164EF9A
:1058C0002CF0000172EF2CF0D890030199379A3731
:1058D0009B379C37D8900336023601369E3700013D
:1058E000DCEF2BF003019EB103D0000180EF2CF020
:1058F000D8900132023203329E33000184EF2CF043
:105900000006D8B4F9EF2CF003019EAF03D00001DC
:10591000D5EF2CF0D89099379A379B379C370001F8
:1059200003019851995FD8A003D00001ACEF2CF08F
:10593000010E9A5FD8A003D00001ACEF2CF09B5F62
:10594000D8A003D00001ACEF2CF09C5FD8B003D0FE
:105950000001E8EF2CF00001030197519A5FD8A0F5
:1059600003D00001C2EF2CF0010E9B5FD8A003D042
:105970000001C2EF2CF09C5FD8B003D00001E8EF2B
:105980002CF00001030196518009000103019B5F87
:10599000D8A003D00001D5EF2CF0010E9C5FD8B049
:1059A00003D00001E8EF2CF00001032AD8A4E8EFAF
:1059B0002CF0022AD8A4E8EF2CF0012AD8A4E8EFB2
:1059C0002CF0002AD8B4F9EF2CF001320232033265
:1059D00092C39DF3030196519D1B9DBF03D000010F
:1059E000F6EF2CF0018E0001FDEF2CF0019EFDEF93
:1059F0002CF0006A016A026A036A000C8E0E006EC7
:105A000003018A51005E8BC302F08CC301F0028E49
:105A10000052D8A403D000011DEF2DF00001D89052
:105A20000252D8A418EF2DF00152D8B41DEF2DF07A
:105A300002320132002E0FEF2DF003018BBF03D095
:105A4000000129EF2DF00001011E021E012AD8B429
:105A5000022A000C03018A51D8A403D00001CAEF26
:105A60002DF0006E8E51D8A403D00001CAEF2DF0A6
:105A70000026D8B003D0000146EF2DF00001810EC2
:105A80000026D8B0CAEF2DF04EEF2DF07F0E005E4D
:105A9000D8A0CAEF2DF0D8B4CAEF2DF08BC392F383
:105AA00003018F51921B8B8F8F8F8D519103F4CFF8
:105AB00094F38C519003F4CF03F0F3CF93F391035D
:105AC000F3509427F4509323000E03228D5190033A
:105AD000F3509427F4509323000E026A032202220B
:105AE0008B519103F3509327F4500322000E0222AE
:105AF0008B519003F3500326F4500222000E016AEA
:105B000001228D518F03F3509327F4500322000E8E
:105B1000022201228C518F03F3500326F4500222FB
:105B2000000E01228B518F03F3500226F450012204
:105B3000002A01AE03D00001A4EF2DF09337033605
:105B40000236013600060001000E030193BF03D0A8
:105B50000001C2EF2DF0032A022201220150D8B425
:105B600003D00001C2EF2DF00250D8B403D00001E1
:105B7000C2EF2DF00350D8B403D00001C2EF2DF0D6
:105B8000002A0001030192BF018E92AF019E000125
:105B9000CEEF2DF0006A016A026A036A000C38C376
:105BA00092F337C391F379EC2BF003C048F302C0B2
:105BB00047F301C046F300C045F33AC392F339C33B
:105BC00091F379EC2BF003C04CF302C04BF301C00E
:105BD0004AF300C049F30301946B240E936F740ED3
:105BE000926F920E916F48C398F347C397F346C3E1
:105BF00096F345C395F300019BEC2BF003C050F3E3
:105C000002C04FF301C04EF300C04DF350C38DF3FB
:105C10004FC38CF34EC38BF34DC38AF3FEEC2CF0D1
:105C200002C03EF301C03DF3036A355003013D5FFE
:105C300003503E5B3AC392F339C391F3000179EC10
:105C40002BF000C051F301C052F302C053F303C064
:105C500054F354C38DF353C38CF352C38BF351C32A
:105C60008AF348C391F347C390F346C38FF345C308
:105C70008EF32AEC2DF000C055F301C056F302C09C
:105C800057F303C058F358C394F357C393F356C361
:105C900092F355C391F30301986B976B7A0E966F4D
:105CA000880E956F00019BEC2BF003C08DF302C0B2
:105CB0008CF301C08BF300C08AF3FEEC2CF002C021
:105CC00040F301C03FF303013C6B3B6B0001030158
:105CD0003C51405DD8B003D00001ACEF2EF0000184
:105CE000D8A47CEF2EF003013F513B5DD8A003D038
:105CF0000001ACEF2EF000018D8635C0C6F3C6C39F
:105D000034F0020E345E00000000000000000000CD
:105D10000000342E87EF2EF08D963EC352F33DC324
:105D200051F3030E0301515F000E525B51C334F077
:105D30005251036A336E332A000100000000342EF2
:105D40009DEF2EF0332E9FEF2EF003013B2BD8B4A6
:105D50003C2B000167EF2EF015EC2BF0000C81506E
:105D6000070B816E070E9316090EC16E820EC06E70
:105D7000090EC26EC290000E016E71EF4FF003016A
:105D8000456B0001030145510708D8B003D000015D
:105D900000EF2FF00001D89003014535476B466FA7
:105DA000820E4625E96E010E4721EA6E4351EF5CF3
:105DB000D8B403D00001FBEF2EF00001D89003010E
:105DC00045354A6B496F010E4925016E000E4A2187
:105DD000036E0150820FE96E010E0320EA6E4451FA
:105DE000EF5CD8B403D00001FBEF2EF00001010EF0
:105DF000016E61EF2FF00301452B0001C2EF2EF081
:105E00000301456B0001030145510708D8B003D0D9
:105E100000015FEF2FF00001D89003014535476B7B
:105E2000466F820E4625E96E010E4721EA6EEF525B
:105E3000D8B403D000015AEF2FF00001D89003012D
:105E400045354A6B496F010E4925016E000E4A2106
:105E5000036E0150820FE96E010E0320EA6EEF52CD
:105E6000D8B403D000015AEF2FF00001D8900301FD
:105E70004535476B466F820E4625E96E010E472178
:105E8000EA6E43C3EFFFD8904535476B466F010E6E
:105E90004625016E000E4721036E0150820FE96E08
:105EA000010E0320EA6E44C3EFFF010E016E0001F4
:105EB00061EF2FF00301452B000103EF2FF0000EDF
:105EC000016E000CA50E0301436F0E0E446F00011E
:105ED000BFEC2EF001C038F303013851016E000110
:105EE000A4EF2FF00301376B0001030137510708BE
:105EF000D8B003D00001A1EF2FF00001D89003012A
:105F00003735396B386F820E3825E96E010E39212D
:105F1000EA6EEF6AD8903735396B386F010E382545
:105F2000016E000E3921036E0150820FE96E010EE1
:105F30000320EA6EEF6A00010301372B000175EFC1
:105F40002FF01E9C62EF2FF00150016E000CCAEC86
:105F500010F0C6EF32F02F6A0301316B000103012C
:105F600031510708D8B003D00001C9EF2FF000016C
:105F7000196AF2BE198EF29E31C3B2F32AEC18F000
:105F800019BEF28E01502F1A0301312B0001AFEF21
:105F90002FF02F52D8A4CFEF2FF08D0E2F6E2FC0E1
:105FA00045F013EF30F0979A9898949A98849594C6
:105FB0009592979A8E9A98988F988C9498968F86A7
:105FC000850ECD6ECD9E080E016E01500409CA6E7D
:105FD000130ECB6ECD96040E6F6E6C946C886C8E27
:105FE0006C9C6B8E6B9A6B9C6B986C9A6B9E196A0F
:105FF000F2BE198EF29E0401146B000129EC04F02C
:1060000019BEF28E326AC950206E3250C96EC7A0D6
:1060100007EF30F0326AC950206E3250C96E8B9A49
:10602000C69AABEF2FF0800E376E010E396E500E10
:106030003A6E020E436E200E426E3D6A3C6A416A21
:10604000246A24500808D8A031EF30F0036A2450A5
:10605000470FE96E000E0320EA6EEF6A242A21EF53
:1060600030F00101966B0001AAEF32F00301476B9B
:10607000486B0001030148510608D8B003D0000165
:1060800061EF30F0000146C303F003014551E96EB2
:1060900003C0EAFFEF504719F2CF4AF3F29E000126
:1060A00053EC00F003014ABFF28E016E01C047F3CA
:1060B000452BD8B4462B00010301482B00013AEFD1
:1060C00030F046C303F003014551E96E03C0EAFF17
:1060D0004751EF5CD8B403D0000176EF30F00001F7
:1060E000010E016E7AEF30F07AEF30F0000E016EA3
:1060F0007AEF30F008EF32F0030145518F08D8A055
:1061000003D0000189EF30F00001000E016E05EFB1
:1061100031F00301465145258F08D8A003D0000176
:1061200097EF30F00001000E016E05EF31F0196AB3
:10613000F2BE198EF29EA1EC18F019BEF28E01C0CB
:1061400049F3196AF2BE198EF29ECC0E0301C46F98
:1061500000011CEC19F019BEF28E196AF2BE198EFC
:10616000F29EF00E0301C46F00011CEC19F019BE81
:10617000F28E196AF2BE198EF29E45C3C4F31CEC6E
:1061800019F019BEF28E196AF2BE198EF29E030141
:10619000C46B00011CEC19F019BEF28E03014A6BAE
:1061A0000001030146514A5DD8A003D00001FAEF77
:1061B00030F0000148C303F0030147514B6F03C0A7
:1061C0004CF3196AF2BE198EF29E00018BEC19F0A5
:1061D00019BEF28E4CC3EAFF4BC3E9FF01C0EFFFCB
:1061E0000301472BD8B4482B000103014A2B0001BF
:1061F000D1EF30F0196AF2BE198EF29EA1EC18F0C0
:1062000019BEF28E03014951016E000115EF32F003
:10621000030E0301446F3B0E436F196AF2BE198EE1
:10622000F29E0001A1EC18F019BEF28E01C039F304
:10623000196AF2BE198EF29E330E0301C46F00017B
:106240001CEC19F019BEF28E44C303F00301435154
:10625000456F03C046F3196AF2BE198EF29E000123
:106260008BEC19F019BEF28E46C3EAFF45C3E9FF75
:1062700001C0EFFF0301432BD8B4442B44C303F008
:106280004351456F03C046F3196AF2BE198EF29E60
:1062900000018BEC19F019BEF28E46C3EAFF45C32C
:1062A000E9FF01C0EFFF0301432BD8B4442B44C3E3
:1062B00003F04351456F03C046F3196AF2BE198ECD
:1062C000F29E00018BEC19F019BEF28E46C3EAFF74
:1062D00045C3E9FF01C0EFFF0301432BD8B4442BB2
:1062E00044C303F04351456F03C046F3196AF2BE3D
:1062F000198EF29E00018BEC19F019BEF28E46C386
:10630000EAFF45C3E9FF01C0EFFF0301432BD8B407
:10631000442B44C303F04351456F03C046F3196A4D
:10632000F2BE198EF29E00018BEC19F019BEF28EAE
:1063300046C3EAFF45C3E9FF01C0EFFF0301432B5A
:10634000D8B4442B44C303F04351456F03C046F314
:10635000196AF2BE198EF29E00018BEC19F019BE7B
:10636000F28E46C3EAFF45C3E9FF01C0EFFF030118
:10637000432BD8B4442B44C303F04351456F03C0AF
:1063800046F3196AF2BE198EF29E00018BEC19F0E9
:1063900019BEF28E46C3EAFF45C3E9FF01C0EFFF15
:1063A0000301432BD8B4442B44C303F04351456F3E
:1063B00003C046F3196AF2BE198EF29E00018BECFF
:1063C00019F019BEF28E46C3EAFF45C3E9FF01C0CA
:1063D000EFFF0301432BD8B4442B196AF2BE198E88
:1063E000F29E0001A1EC18F019BEF28E080E030116
:1063F000435F000E445B3953D8A403D000010AEF79
:1064000032F0000144C346F343C345F336EF30F0A6
:1064100001C039F30301456B020E466F38C348F3E0
:1064200037C347F300017CEF30F0060E030143272A
:10643000000E4423020E3727000E38233953D8A408
:1064400003D0000155EF32F0000103013A6B000167
:1064500003013A510508D8B003D0000153EF32F0E0
:10646000000138C303F003013751456F03C046F301
:1064700044C303F04351E96E03C0EAFFEF50476F96
:1064800046C3EAFF45C3E9FF47C3EFFF372BD8B444
:10649000382B4351D8B444074307000103013A2B7A
:1064A000000128EF32F073EF32F0020E03013A6F71
:1064B000000103013A510708D8B003D0000173EF7F
:1064C00032F0000138C303F003013751E96E03C015
:1064D000EAFFEF6A372BD8B4382B000103013A2BBF
:1064E000000159EF32F003013951016E000184EFD0
:1064F00032F08D9C88EF32F020EC2BF035C338F36E
:1065000034C337F308EF31F001C036F379EF32F0DE
:1065100003013651016E000196EF32F0010E0301C6
:10652000356F240E346F00017CEF32F001C032F37E
:1065300003013251016E0001ACEF32F0526A050ED8
:106540000101216F516A1E961E98030E406F0001D3
:10655000D3EF2FF08EEF32F08CEF33F0196AF2BEEA
:10656000198EF29E2FEC10F019BEF28E9CEC18F0F2
:1065700072EC2FF01E9A0101926B1E9C1E8E93915D
:106580009393816B926B0001A7EF2FF0196AF2BE13
:10659000198EF29E010E0301AE6F00018DEC18F012
:1065A00019BEF28E9CEC18F00301C46BC80EC36FC9
:1065B00000010301C351C411D8A403D000012EEF80
:1065C00033F00001FA0E0301C66F0001C6C334F0B8
:1065D000020E345E00000000000000000000000019
:1065E000342EEEEF32F0FA0E0301C66F0001C6C37F
:1065F00034F0020E345E00000000000000000000D5
:106600000000342EFFEF32F0FA0E0301C66F0001D6
:10661000C6C334F0020E345E00000000000000002B
:1066200000000000342E10EF33F0FA0E0301C66FA5
:106630000001C6C334F0020E345E0000000000000A
:10664000000000000000342E21EF33F00301C3519D
:10665000D8B4C407C3070001D9EF32F016EC10F02C
:106660000301C46BC80EC36F00010301C351C41101
:10667000D8A403D000018AEF33F00001FA0E030121
:10668000C66F0001C6C334F0020E345E0000000085
:106690000000000000000000342E4AEF33F0FA0E34
:1066A0000301C66F0001C6C334F0020E345E000061
:1066B00000000000000000000000342E5BEF33F00B
:1066C000FA0E0301C66F0001C6C334F0020E345E39
:1066D000000000000000000000000000342E6CEFFD
:1066E00033F0FA0E0301C66F0001C6C334F0020E88
:1066F000345E000000000000000000000000342EA6
:106700007DEF33F00301C351D8B4C407C3070001C0
:1067100035EF33F09EEF32F0196AF2BE198EF29E19
:10672000B6EC1CF019BEF28E73EF4FF0010193919D
:10673000030130A103D0010193810301010193936F
:10674000030131A103D0010193830301000199EFFB
:106750004FF09688050E006E002EACEF33F0968A4F
:10676000060E006E002EB2EF33F08D989698050E4F
:10677000006E002EB9EF33F08D9A969A000C080E39
:10678000016E050E006E002EC3EF33F08D9A969ABF
:10679000060E006E002ECAEF33F0030135378D98D8
:1067A000D8B09688D8A09698968A000184AAD6EF89
:1067B00033F0012EC1EF33F0050E006E002EDEEF38
:1067C00033F08D9A969A00009688060E006E002E81
:1067D000E7EF33F0060E006E002EECEF33F0968AF2
:1067E00084AAF0EF33F0016A060E006E002EF6EF79
:1067F00033F084B801808D9A969A8D98969805EF1B
:1068000034F034C335F3BFEF33F00150016E000CA8
:1068100096980000968A84AA0BEF34F0050E006E5D
:10682000002E10EF34F000D000009688050E006EA8
:10683000002E18EF34F0000C030EEA6E450EE96EE0
:10684000EF50D8B431EF34F0060E016E006A002E1E
:10685000FED7012EFBD77B0E006E002EFED7EF2E4B
:10686000F3D7000C080E0301366F00C037F30001A8
:106870009688060E006E002E3BEF34F0968A84AAAE
:106880003FEF34F084B8D88084A8D8900136050E44
:10689000006E002E49EF34F0969A8D9A0301362F40
:1068A00002D004D00001000138EF34F09688060EC3
:1068B000006E0001002E5AEF34F08D98030137511D
:1068C000D8A4969800010000968A84AA65EF34F057
:1068D000050E006E002E6AEF34F08D9A969A060E21
:1068E000006E002E71EF34F08D9896987CEF34F0A6
:1068F00034C300F032EF34F00150016E000C800E12
:106900000301336F326B0001A9EC33F0900E0301E9
:10691000346F000101EC34F00152D8A498EF34F048
:10692000EE0E0301346F000101EC34F008EC34F09A
:10693000040E0301346F0001FA0E0301456F0001DC
:106940001CEC34F00301342F02D003D0000100010D
:10695000F3D70001A9EC33F0900E0301346F00016E
:1069600001EC34F00152D8A4FEEF34F0AA0E03017A
:10697000346F000101EC34F00152D8B4C0EF34F0B0
:10698000800E0301336F326B0001A9EC33F0910EDE
:106990000301346F000101EC34F00152D8A4FEEF82
:1069A00034F00301346B000178EC34F001C030F3B3
:1069B0000301346B000178EC34F001C031F330C3D3
:1069C00033F331C332F303013333323333333233EE
:1069D000333332333333323333333233333332338B
:1069E00033333233010E331730BF03D00001FEEFD3
:1069F00034F00001FE0E03013313000108EC34F003
:106A000003013251016E3351026E0001BEEF4FF0AF
:106A1000030167513C24686F000E3D20696F00013F
:106A2000030168513C5CD8B403D0000110EF35F08D
:106A30000001030169513D5CD8B403D0000110EF9F
:106A400035F00001000C1EA82AEF35F0010E016E92
:106A50002CEF35F0000E016E30EF35F023EF35F0FE
:106A60000150016E000C0301476B0001020E010191
:106A7000165D0301475DD8A403D0000146EF35F051
:106A8000D8A003D000017AEF35F00001036A0301BA
:106A90004751550FE96E000E0320EA6E4551EF5C39
:106AA000D8B403D0000175EF35F00001010E0301E9
:106AB0004725036A550FE96E000E0320EA6E465122
:106AC000EF5CD8B403D0000175EF35F00001020E81
:106AD00003014725036A550FE96E000E0320EA6E95
:106AE000EF50016E00017CEF35F00301472B0001F0
:106AF00036EF35F0FF0E016E000C43C345F344C37F
:106B000046F333EC35F00150FF08D8B48EEF35F082
:106B1000010E016E92EF35F092EF35F0000E016E2E
:106B200092EF35F0000C0301456B0001020E0101EC
:106B3000165D0301455DD8A403D00001A6EF35F032
:106B4000D8A003D00001EBEF35F00001036A030188
:106B50004551550FE96E000E0320EA6E4351EF5C7C
:106B6000D8B403D00001E6EF35F00001010E0301B7
:106B70004525036A550FE96E000E0320EA6E445165
:106B8000EF5CD8B403D00001E6EF35F00001020E4F
:106B900003014525036A550FE96E000E0320EA6ED6
:106BA000EF52D8A403D00001E6EF35F00001030E48
:106BB00003014525036A550F016E000E03220150A3
:106BC000016E0350026E0001EBEF35F00301452B1F
:106BD000000196EF35F0000C030E0301465FD8B0BC
:106BE00003D0000104EF36F0030EEA6E460EE96EA4
:106BF000EF50D8A403D0000104EF36F0000102EFFB
:106C000036F000D0EF2EFDD748EF36F00301376B9A
:106C1000386B396B3A6B3D6B3E6B3F6B406B416B36
:106C2000426B436B446B3351E96E3451EA6EEC6A4C
:106C3000ED52EF6A020E3325E96E000E3421EA6E42
:106C4000EC6AED52EF6A040E3325E96E000E342132
:106C5000EA6EEC6AED52EF6A060E3325E96E000E1D
:106C60003421EA6EEC6AED52EF6A8150070B816EB7
:106C70008A96030E456F00011CEC34F0020E0301EE
:106C8000456F0001F90E0301466F0001ECEF35F08E
:106C90000301452F02D003D000010001F3D7090EF4
:106CA000C26E170E006E0001002EFED703013A518E
:106CB0000108D8B003D0000138EF37F00001D8A4A4
:106CC0006BEF36F0030139518F08D8B003D00001C3
:106CD00038EF37F00001C282C2B26CEF36F0196AA9
:106CE000F2BE198EF29E0301F46BC4CFF3F3010ED2
:106CF000F66FF56B000119EC09F019BEF28E02C0B7
:106D000046F301C045F3C350030145253B6F000E18
:106D100046213C6FD8903835036A3D0F016E030E53
:106D200003220150456F03C046F3D8903835036AFB
:106D30003D0FE96E030E0320EA6EECCF48F3ED52EF
:106D4000EFCF47F33B514725016E3C514821036E7D
:106D50000150496F03C04AF346C3EAFF45C3E9FF48
:106D60004AC3ECFFED5249C3EFFFD8903835036AB0
:106D70003325E96E34510320EA6EECCF03F0ED5277
:106D8000EF50016E03503C5DD8B003D00001E5EF39
:106D900036F00001D8A4D6EF36F003013B51015C78
:106DA000D8A003D00001E5EF36F00001D890030130
:106DB0003835036A3325E96E34510320EA6E3CC34B
:106DC000ECFFED523BC3EFFF000103013851020815
:106DD000D8A003D00001F3EF36F000010301386BB7
:106DE0000001F6EF36F00301382B000103013853A0
:106DF000D8B403D0000102EF37F00001090EC26ED3
:106E00002DEF37F00301382D02D004D0000100012E
:106E10000FEF37F000010D0EC26E2DEF37F00301BA
:106E200038510208D8B403D000011CEF37F000013C
:106E3000150EC26E2DEF37F0030138510308D8B498
:106E400003D0000129EF37F00001110EC26E2DEFC3
:106E500037F0FF0E016E19EF38F0170E006E002E9E
:106E6000FED70301392BD8B43A2B000156EF36F088
:106E7000C2900301426B416B040E3325E96E000E94
:106E80003421EA6EEC6AED52EF6A376B00010301C0
:106E900037510308D8B003D0000117EF38F00001D4
:106EA000D89003013735036A3125016E3251032230
:106EB0000150456F03C046F3D8903735036A3D0F44
:106EC000E96E030E0320EA6EECCF48F3ED52EFCFEC
:106ED00047F3196AF2BE198EF29E48C3EEF347C318
:106EE000EDF3F06B640EEF6F000101EC11F019BED1
:106EF000F28E02C003F001500301486F03C049F352
:106F000046C3EAFF45C3E9FF49C3ECFFED5248C35E
:106F1000EFFFD8903735036A3525016E36510322CD
:106F20000150456F03C046F3D8903735036A3325C7
:106F3000E96E34510320EA6EECCF48F3ED52EFCF07
:106F400047F3D8903735036A3125E96E3251032073
:106F5000EA6EECCF03F0ED52EF50475D496F0350FE
:106F600048594A6F196AF2BE198EF29E4AC3F4F369
:106F700049C3F3F3F66B8C0EF56F000119EC09F0C1
:106F800019BEF28E02C04BF301C04AF3196AF2BE79
:106F9000198EF29E4BC3EEF34AC3EDF30301F06B7F
:106FA000640EEF6F000101EC11F019BEF28E02C009
:106FB00003F0015003014B6F03C04CF346C3EAFFDB
:106FC00045C3E9FF4CC3ECFFED524BC3EFFFD89034
:106FD0003735036A3525E96E36510320EA6EECCF6A
:106FE00046F3ED52EFCF45F34653D8B403D000013A
:106FF00012EF38F00001030145510508D8B003D065
:10700000000112EF38F00001D89003013735036A10
:107010003525E96E36510320EA6EEC6AED52060E14
:10702000EF6E00010301372B000147EF37F0000E30
:10703000016E89EF38F0640E0301306F196AF2BEF9
:10704000198EF29E0001B6EC1CF019BEF28E0301FF
:107050003053D8A403D0000171EF38F00001010EC5
:107060000301676F000108EC35F02EEC35F001529A
:10707000D8B46CEF38F0750E0301436F660E446FA1
:1070800000017DEC35F00152D8B46CEF38F0750E8C
:107090000301456F660E466F000133EC35F0012C9D
:1070A0006CEF38F0750E0301436F660E446F0001FC
:1070B00093EC35F002C003F00150E96E03C0EAFF23
:1070C000EF52D8A46CEF38F0050E0301676F000192
:1070D00008EC35F071EF38F003013007000127EFBD
:1070E00038F0196AF2BE198EF29E2FEC10F019BE1C
:1070F000F28E020E0301326FE60E316F020E346F14
:10710000EE0E336F020E366FF60E356F000106EF8E
:1071100036F08AEF50F01EAA92EF38F0020E016EA0
:10712000CAEF38F0400ED880010181550208D8B06E
:1071300003D00001A3EF38F00001010E016ECAEF89
:1071400038F0CAEF38F0036A01018151410FE96E4E
:10715000010E0320EA6E47C3EFFF010E8125036A8B
:10716000410FE96E010E0320EA6E48C3EFFF020EE5
:107170008125036A410FE96E010E0320EA6EEF6A72
:10718000020E8125926F030E8127000E016E000111
:10719000CAEF38F0000C1EAAD2EF38F0020E016ED2
:1071A000FCEF38F0400ED88001018155000AD8B4B8
:1071B00003D00001E3EF38F00001010E016EFCEF97
:1071C00038F0FCEF38F0036A01019251410FE96E8B
:1071D000010E0320EA6EEF2A036A8151410FE96E26
:1071E000010E0320EA6E48C3EFFF010E8127000E57
:1071F000016E0001FCEF38F0000C37BE04EF39F0EF
:10720000000E016E37EF39F037A00BEF39F0000EAA
:10721000016E37EF39F0EA6A950EE96E010EE26E03
:10722000410EE16E400E016EE6CFEEFF012E14EF2F
:1072300039F081C151F0196AF2BE198EF29E47C32E
:10724000E9F323EC16F019BEF28E0152D8B433EFF5
:1072500039F00101816B926B010E016E000137EF75
:1072600039F037EF39F0000E016E37EF39F0000CCE
:10727000750E0301476F660E486F00018BEC38F006
:107280007B0E0301476F0E0E486F00018BEC38F048
:10729000010E0301486F0001CBEC38F03E0E0301F4
:1072A000486F0001CBEC38F0E3C230F330C348F351
:1072B000CBEC38F0E2C230F330C348F3CBEC38F01B
:1072C000E5C230F330C348F3CBEC38F0E4C230F31E
:1072D00030C348F3CBEC38F0E7C230F330C348F3A7
:1072E000CBEC38F0E6C230F330C348F3CBEC38F0E7
:1072F000E9C230F330C348F3CBEC38F0E8C230F3E6
:1073000030C348F3CBEC38F0EBC230F330C348F372
:10731000CBEC38F0EAC230F330C348F3CBEC38F0B2
:10732000EDC230F330C348F3CBEC38F0ECC230F3AD
:1073300030C348F3CBEC38F0EFC230F330C348F33E
:10734000CBEC38F0EEC230F330C348F3CBEC38F07E
:10735000F1C230F330C348F3CBEC38F0F0C230F375
:1073600030C348F3CBEC38F0F3C230F330C348F30A
:10737000CBEC38F0F2C230F330C348F3CBEC38F04A
:10738000F5C230F330C348F3CBEC38F0F4C230F33D
:1073900030C348F3CBEC38F0F7C230F330C348F3D6
:1073A000CBEC38F0F6C230F330C348F3CBEC38F016
:1073B000F9C230F330C348F3CBEC38F0F8C230F305
:1073C00030C348F3CBEC38F0FBC230F330C348F3A2
:1073D000CBEC38F0FAC230F330C348F3CBEC38F0E2
:1073E000FDC230F330C348F3CBEC38F0FCC230F3CD
:1073F00030C348F3CBEC38F0140E0301476F0001A3
:10740000FDEC38F0196AF2BE198EF29E04EC22F0FF
:1074100019BEF28E0152D8B416EF3AF0010E0301F4
:10742000676F000108EC35F002EF3AF094EF50F08E
:1074300003013951000A0001D8B421EF3AF026EFD8
:107440003AF0CD86770EB16E26EF3AF02CEF3AF097
:1074500038C339F318EF3AF0EFEF3BF047C3B3FF0F
:1074600036EF3AF046C347F32EEF3AF048EF3AF0E2
:1074700047C3B2FF40EF3AF046C347F338EF3AF064
:107480004CEF3AF043C329F344C346F332EF3AF0EA
:1074900045C346F33CEF3AF044C32AF3000C37A24D
:1074A00058EF3AF0010E016E5CEF3AF05CEF3AF003
:1074B000000E016E5CEF3AF060EF3AF04FEF3AF0F9
:1074C0000152D8B46AEF3AF0010E016E6EEF3AF055
:1074D0006EEF3AF0000E016E6EEF3AF0000C030111
:1074E0004291010E3B6F5E0E3A6F3D6B100E3C6F8A
:1074F000D30E436F370E446F0001BFEC2EF0030133
:107500003BAF03D00001E2EF3BF03B53D8B403D0D4
:10751000000195EF3AF0000103013A510008D8A0AC
:1075200003D00001E2EF3BF000012EEC35F00152F8
:10753000D8B4D1EF3BF0750E0301436F660E446F74
:1075400000017DEC35F00152D8B4D1EF3BF0D30E01
:107550000301436F370E446F00017DEC35F001529B
:10756000D8B409EF3BF0D30E0301436F370E446FDD
:10757000000193EC35F002C039F301C038F3020E7C
:1075800003013825E96E000E3921EA6E400EEF2422
:107590003F6F010E3825E96E000E3921EA6EEF507B
:1075A000406F3851E96E3951EA6EEF50416F020E6B
:1075B0003825E96E000E3921EA6EEF503F5DD8A004
:1075C00003D00001E8EF3AF000010301402B000175
:1075D000010E03013825E96E000E3921EA6EEF50E5
:1075E000405DD8A003D00001FAEF3AF0000103019A
:1075F000412B000141C343F340C344F33FC345F370
:1076000042EC3AF0030142810001E2EF3BF0D1EF9E
:107610003BF003013D53D8B403D000011AEF3BF017
:10762000000103013C510F08D8A003D00001D1EFA5
:107630003BF000010F0E03013E6F00012EEC35F010
:107640000152D8B46DEF3BF0750E0301436F660E27
:10765000446F00017DEC35F00152D8B46DEF3BF082
:10766000750E0301456F660E466F000133EC35F071
:10767000012C6DEF3BF0750E0301436F660E446FF6
:10768000000193EC35F002C003F00150E96E03C035
:10769000EAFFEF52D8A45FEF3BF0040E0301676FDF
:1076A000000108EC35F0040E03013A5F000E3B5B6D
:1076B000040E3E5F040E3C27000E3D230001C60E63
:1076C0000301476FB70E486F00018BEC38F0010ED5
:1076D0000301476F0001FDEC38F0010E0301676FF5
:1076E000000108EC35F003013A51D8B43B073A07E2
:1076F0003E073C2BD8B43D2B00012EEC35F0015257
:10770000D8B49DEF3BF0750E0301436F660E446FD6
:1077100000017DEC35F00152D8B49DEF3BF0D30E63
:107720000301436F370E446F00017DEC35F00152C9
:10773000D8B49DEF3BF0B3EF3AF05EEC3AF0015273
:10774000D8B4B3EF3BF0196AF2BE198EF29E7AEC10
:1077500021F019BEF28E0152D8B4B3EF3BF0030111
:107760003D6B3C6B000103013C53D8B403D00001D6
:10777000C3EF3BF0000103013D53D8A403D0000147
:10778000D1EF3BF0000103013EAF03D00001D1EF88
:107790003BF03E510008D8B003D000011EEF3BF093
:1077A0000001010E0301676F000108EC35F00301D1
:1077B0003A51D8B43B073A073C2BD8B43D2B0001D3
:1077C0007FEF3AF0000E030142B1010E016E00019D
:1077D000F8EF3BF00301386B000128EF3AF0530E4D
:1077E000006E002EFED70201FE9500016FEF3AF009
:1077F00001B000EF3CF003013791000103EF3CF0D2
:10780000030137810001030137A103D0000111EF0B
:107810003CF000010301436B446B456B000142ECFB
:107820003AF0000E030137B1010E016E000112EFB4
:107830004DF003014B51016A4A5DD8A003D000010D
:1078400027EF3CF04A51006E00013BEF3CF0006A2C
:10785000080E03014C6F000103014A3700364B51FB
:10786000005CD8B0006E01364C2F02D004D000016D
:1078700000012CEF3CF00001000C010E03012B6F06
:10788000D8902835070F376F0001030137514008A2
:10789000D8A003D0000161EF3CF0000103012B2BC5
:1078A000400E375F37B103D000015BEF3CF00001C1
:1078B0000301372B0001070E03013727000145EFB5
:1078C0003CF0010E03012C6F2851060DF350070FF9
:1078D000386F0001030138514008D8A003D00001DF
:1078E00086EF3CF0000103012C2B400E385F38C3BB
:1078F0004AF3060E4B6F000119EC3CF000500301F7
:107900003827070E382700016AEF3CF003012C519D
:107910002B252D6F040E2D25010F2E6F2F6B285355
:10792000D8A403D00001ABEF3CF00001196AF2BE0D
:10793000198EF29E2FC3F4F32EC3F3F30301F66BFB
:1079400028C3F5F3000119EC09F019BEF28E02C04C
:107950002FF301C02EF3000C0301376B000103016C
:1079600037513208D8B003D00001DFEF3CF00001FE
:10797000036A03013751AC0FE96E010E0320EA6E72
:10798000EFCF38F3AA6A37C3A9FF38C3A8FFA69C74
:10799000A69EA684F250006EF29E0F01550EA76EB1
:1079A000AA0EA76EA6820001A6B2D4EF3CF0A69460
:1079B0000050F2120301372B0001AFEF3CF0000E34
:1079C000016EF2EF4DF0196AF2BE198EF29E98EC3C
:1079D00027F019BEF28E01C068F3196AF2BE198E43
:1079E000F29EA0EC27F019BEF28E01C067F30301EE
:1079F00068BF03D0000101EF3DF000010301672BD8
:107A0000000103016751016E0001000C0301419167
:107A10000101DF5103013E5DD8A403D000017AEFDC
:107A20003DF00001E3EC3CF003013F51015C3F08F5
:107A3000D8B003D000017AEF3DF000010301406BA4
:107A4000000103012851405DD8A003D000015DEF83
:107A50003DF00001036A03014051E96E030E032467
:107A6000EA6EEF503E5DD8B403D0000158EF3DF010
:107A70000001036A03014051140FE96E030E032055
:107A8000EA6EEF503F5D3F08D8B003D0000155EFDC
:107A90003DF00001036A03014051140FE96E030E2B
:107AA0000320EA6E3FC3EFFF0001030141810001A3
:107AB0000301402B000121EF3DF0030141A103D060
:107AC00000017AEF3DF00001036A03012851E96EDD
:107AD000030E0324EA6E3EC3EFFF036A2851140F1E
:107AE000E96E030E0320EA6E3FC3EFFF282B0A0E58
:107AF0000201FF6F0001000CCB0E0301456F810EE8
:107B0000466F000133EC35F001C038F3CB0E0301B2
:107B1000436F810E446F000193EC35F002C03AF3DD
:107B200001C039F30301376B000103013851375DA0
:107B3000D8A003D00001BFEF3DF00001036A0301AC
:107B400037513925E96E3A510320EA6EEFCF3BF306
:107B5000010E3725036A3925E96E3A510320EA6E92
:107B6000EFCF3DF33BC33EF33DC33FF3000106ECD3
:107B70003DF0020E03013727000195EF3DF060EF65
:107B80004EF00201FE830001E3EC3CF001C039F34A
:107B90000301376B000103012851375DD8A003D0E2
:107BA00000014AEF3EF00001036A03013751140F50
:107BB000E96E030E0320EA6EEF50395D3F08D8A04E
:107BC00003D0000132EF3EF00001010E0301372522
:107BD000386F000103012851385DD8A003D000019F
:107BE0002CEF3EF00001010E0301385D036A016EC7
:107BF000030E032601503B6F03C03CF3036A385168
:107C0000E96E030E0324EA6EEF503D6F3CC3EAFFBA
:107C10003BC3E9FF3DC3EFFF010E385D036A140F5C
:107C2000016E030E032201503B6F03C03CF3036A55
:107C30003851140FE96E030E0320EA6EEF503D6FCA
:107C40003CC3EAFF3BC3E9FF3DC3EFFF0001030173
:107C5000382B0001EAEF3DF0030128073707000148
:107C600045EF3EF0036A03013751E96E030E03242A
:107C7000EA6EEF500101DF5DD8A003D0000145EFAF
:107C80003EF000010201FE9300010301372B0001C9
:107C9000CBEF3DF06CEF4EF067C339F0000C379836
:107CA00054EF3EF04FEF3EF0000C03016D6B00010E
:107CB00003016D510308D8B003D00001DCEF3EF0A2
:107CC0000001D89003016D35036A6B25E96E6C5194
:107CD0000320EA6EECCF6FF3ED52EFCF6EF3D89046
:107CE0006D35036A6925E96E6A510320EA6EECCFAF
:107CF00003F0ED52EF50016E03506F5DD8B003D02A
:107D00000001CAEF3EF00001D8A490EF3EF003015D
:107D10006E51015CD8A003D00001CAEF3EF0000113
:107D2000D89003016D35036A6725016E68510322FF
:107D300001506E6F03C06FF3D8906D35036A6B25E9
:107D4000E96E6C510320EA6EECCF71F3ED52EFCF88
:107D500070F3D8906D35036A6925E96E6A51032086
:107D6000EA6EECCF03F0ED52EF50705D006E035001
:107D70007159036E0050726F03C073F36FC3EAFF53
:107D80006EC3E9FF73C3ECFFED5272C3EFFF000156
:107D9000D7EF3EF0D89003016D35036A6725E96E91
:107DA00068510320EA6EEC6AED52EF6A00010301AC
:107DB0006D2B000158EF3EF0040E03016725E96EBC
:107DC000000E6821EA6EEC6AED52EF6A000E016E59
:107DD00000010AEF49F003016F6B000103016F51CD
:107DE0000308D8B003D000016BEF3FF00001036A35
:107DF00003016F516D25E96E6E510320EA6EEF6A43
:107E0000D8906F35036A6725E96E68510320EA6EE2
:107E1000ECCF76F3ED52EFCF75F3753D02D004D081
:107E20000001000120EF3FF000010301763D02D088
:107E300004D00001000120EF3FF000015CEF3FF0B3
:107E4000D89003016F35036A6925E96E6A510320F2
:107E5000EA6EECCF78F3ED52EFCF77F3D8906F3531
:107E6000036A6B25E96E6C510320EA6EECCF03F0D8
:107E7000ED52EF50016E0350785DD8B003D0000191
:107E80005CEF3FF00001D8A44FEF3FF003017751C2
:107E9000015CD8A003D000015CEF3FF00001036A51
:107EA00003016F51700FE96E030E0320EA6E010E9D
:107EB000EF6E000166EF3FF0036A03016F51700F30
:107EC000E96E030E0320EA6EEF6A000103016F2BD7
:107ED0000001EEEF3EF0FF0E0301746F6F6B0001C7
:107EE00003016F510308D8B003D00001CBEF3FF07E
:107EF0000001036A03016F51700FE96E030E032046
:107F0000EA6EEF52D8A403D00001C6EF3FF00001A3
:107F10000301743D02D004D00001000195EF3FF051
:107F200000016FC374F3C6EF3FF0D89003016F35C3
:107F3000036A6725E96E68510320EA6EECCF76F399
:107F4000ED52EFCF75F3D8907435036A6725E96E6B
:107F500068510320EA6EECCF03F0ED52EF50016E52
:107F60007651035CD8B003D00001C6EF3FF00001AA
:107F7000D8A4C4EF3FF001500301755DD8A003D031
:107F80000001C6EF3FF000016FC374F303016F2BD4
:107F9000000170EF3FF00301743D02D004D00001F6
:107FA0000001D6EF3FF0000138EF40F003016F6BA6
:107FB000000103016F510308D8B003D0000138EF6E
:107FC00040F00001D89003016F35036A6725E96E20
:107FD00068510320EA6EECCF76F3ED52EFCF75F3E4
:107FE000D8907435036A6725E96E68510320EA6EFC
:107FF000ECCF78F3ED52EFCF77F3E80E7725016EF3
:10800000030E7821036E0150016E7651035CD8B0E7
:1080100003D0000133EF40F00001D8A419EF40F085
:1080200001500301755DD8A003D0000133EF40F08B
:108030000001036A03016F51700FE96E030E032004
:10804000EA6EEF52D8A403D0000133EF40F00001F4
:10805000036A03016F516D25E96E6E510320EA6ECC
:10806000010EEF6E000103016F2B0001D9EF3FF00D
:10807000000E016E20EF49F0020E03016F6F706B6E
:10808000030E716F010E726F010E736F030E746F2A
:10809000756B020E766FB40E776F786B5A0E796F30
:1080A0007A6B0E0E7B6F010E7C6F7D6B7E6B816B2E
:1080B000806B040E7F6F826B000103018251030805
:1080C000D8B003D00001A0EF40F00001D890030128
:1080D0008235036A6725E96E68510320EA6EECCFAA
:1080E00003F0ED52EF50016E8151035CD8B003D024
:1080F00000019BEF40F00001D8A488EF40F0015050
:108100000301805DD8A003D000019BEF40F0000187
:10811000D89003018235036A6725E96E6851032010
:10812000EA6EECCF03F0ED52EF50806F03C081F3A5
:1081300082C37FF300010301822B00015DEF40F059
:1081400003017F510408D8B403D00001C0EF40F010
:1081500000016CC303F003016B51E96E03C0EAFF39
:10816000EC6AED52EF6A6EC303F06D51E96E03C025
:10817000EAFF050EEF6E010E016E0001E8EF43F01D
:108180006EC303F003016D51E96E03C0EAFFEF6AAD
:10819000D8907F35036A770FE96E030E0320EA6EED
:1081A000ECCF03F0ED52EF50876F03C088F3036A02
:1081B0007F516925E96E6A510320EA6EEF2C02D0E7
:1081C00004D000010001AAEF43F000016EC303F0E8
:1081D00003016D51E96E03C0EAFF010EEF6E036A01
:1081E0007F516F0FE96E030E0320EA6E036AEF50B2
:1081F0006925E96E6A510320EA6EEF2C02D004D0A3
:1082000000010001A0EF42F00001036A03017F5169
:10821000730FE96E030E0320EA6E036AEF506925BF
:10822000E96E6A510320EA6EEF2C02D004D00001FF
:108230000001A0EF42F000016EC303F003016D5195
:10824000E96E03C0EAFF030EEF6E036A7F516F0F02
:10825000E96E030E0320EA6ED890EF34036A6725B7
:10826000E96E68510320EA6EECCF8BF3ED52EFCF4D
:108270008AF3036A7F51730FE96E030E0320EA6EDF
:10828000D890EF34036A6725E96E68510320EA6EDF
:10829000ECCF03F0ED52EF50016E03508B5DD8B080
:1082A00003D00001E1EF41F00001D8A461EF41F0FB
:1082B00003018A51015CD8A003D00001E1EF41F035
:1082C0000001036A03017F516F0FE96E030E032063
:1082D000EA6ED890EF34036A6725E96E685103208F
:1082E000EA6EECCF8BF3ED52EFCF8AF3036A7F5146
:1082F000730FE96E030E0320EA6ED890EF34036A21
:108300006725E96E68510320EA6EECCF03F0ED5269
:10831000EF508A5D006E03508B59036E0050916FD1
:1083200003C092F3000179EC2BF000C08DF301C083
:108330008EF302C08FF303C090F381C392F380C326
:1083400091F379EC2BF090C394F38FC393F38EC326
:1083500092F38DC391F303C098F302C097F301C069
:1083600096F300C095F39BEC2BF003C086F302C09C
:1083700085F301C084F300C083F303018D6B8C6B24
:10838000340E8B6F840E8A6F86C391F385C390F38E
:1083900084C38FF383C38EF300012AEC2DF003C056
:1083A0008DF302C08CF301C08BF300C08AF3FEECA6
:1083B0002CF002C003F001500301872703508823EB
:1083C0000001036A03017F51730FE96E030E03205E
:1083D000EA6ED890EF34036A6725E96E685103208E
:1083E000EA6EECCF8BF3ED52EFCF8AF3036A7F5145
:1083F0006F0FE96E030E0320EA6ED890EF34036A24
:108400006725E96E68510320EA6EECCF03F0ED5268
:10841000EF50016E03508B5DD8B003D000019EEF8A
:1084200042F00001D8A41EEF42F003018A51015C22
:10843000D8A003D000019EEF42F00001036A0301BF
:108440007F51730FE96E030E0320EA6ED890EF346C
:10845000036A6725E96E68510320EA6EECCF8BF35F
:10846000ED52EFCF8AF3036A7F516F0FE96E030E6F
:108470000320EA6ED890EF34036A6725E96E6851ED
:108480000320EA6EECCF03F0ED52EF508A5D006EF0
:1084900003508B59036E0050916F03C092F300019B
:1084A00079EC2BF000C08DF301C08EF302C08FF386
:1084B00003C090F381C392F380C391F379EC2BF066
:1084C00090C394F38FC393F38EC392F38DC391F350
:1084D00003C098F302C097F301C096F300C095F370
:1084E0009BEC2BF003C086F302C085F301C084F33C
:1084F00000C083F303018D6B8C6B340E8B6F840E85
:108500008A6F86C391F385C390F384C38FF383C3CB
:108510008EF300012AEC2DF003C08DF302C08CF322
:1085200001C08BF300C08AF3FEEC2CF002C003F014
:1085300001500301875F0350885B0001AAEF43F0FD
:10854000036A03017F516F0FE96E030E0320EA6E89
:10855000036AEF506925E96E6A510320EA6EEF2C39
:1085600002D004D00001000125EF43F000016EC3EA
:1085700003F003016D51E96E03C0EAFF020EEF6ED6
:10858000036A7F516F0FE96E030E0320EA6ED890E5
:10859000EF34036A6725E96E68510320EA6EECCF79
:1085A00003F0ED52EF50916F03C092F3000179ECAC
:1085B0002BF000C08AF301C08BF302C08CF303C020
:1085C0008DF381C392F380C391F379EC2BF08DC3CB
:1085D00094F38CC393F38BC392F38AC391F303C0D8
:1085E00098F302C097F301C096F300C095F39BEC9B
:1085F0002BF003C086F302C085F301C084F300C0F2
:1086000083F303018D6B8C6B340E8B6F840E8A6F3A
:1086100086C391F385C390F384C38FF383C38EF332
:1086200000012AEC2DF003C08DF302C08CF301C0D1
:108630008BF300C08AF3FEEC2CF002C003F0015073
:1086400003018727035088230001036A03017F5138
:10865000730FE96E030E0320EA6E036AEF5069257B
:10866000E96E6A510320EA6EEF2C02D004D00001BB
:108670000001AAEF43F000016EC303F003016D5146
:10868000E96E03C0EAFF020EEF6E036A7F51730FBB
:10869000E96E030E0320EA6ED890EF34036A672573
:1086A000E96E68510320EA6EECCF03F0ED52EF5013
:1086B000916F03C092F3000179EC2BF000C08AF3B4
:1086C00001C08BF302C08CF303C08DF381C392F31E
:1086D00080C391F379EC2BF08DC394F38CC393F3A7
:1086E0008BC392F38AC391F303C098F302C097F34C
:1086F00001C096F300C095F39BEC2BF003C086F30A
:1087000002C085F301C084F300C083F303018D6BC5
:108710008C6B340E8B6F840E8A6F86C391F385C386
:1087200090F384C38FF383C38EF300012AEC2DF002
:1087300003C08DF302C08CF301C08BF300C08AF339
:10874000FEEC2CF002C003F001500301875F0350E0
:10875000885B0001030188AF03D00001B3EF43F051
:108760000001B9EF43F0680E03018727010E88234B
:108770000001030188AF03D00001DAEF43F0885114
:108780000008D8A003D00001DAEF43F00001FF0A8F
:10879000D8A4D4EF43F0030187516708D8A003D0D1
:1087A0000001DAEF43F00001680E0301875F010E5C
:1087B000885B00016CC303F003016B51E96E03C0D9
:1087C000EAFF88C3ECFFED5287C3EFFF000E016E96
:1087D000000136EF49F0030185518719800B896F3D
:1087E00085BF03D00001FBEF43F0841F851F842B5E
:1087F000D8B4852B0001030187BF03D0000107EF28
:1088000044F0861F871F862BD8B4872B0001016A8E
:10881000026A006A036A03018751D8B403D00001D9
:1088200019EF44F08651D8A403D0000144EF44F07E
:108830000001100E0301886F0001D89003018437F6
:108840008537003603368751035CD8B403D0000166
:108850002DEF44F08651005C0001D8A039EF44F0C0
:1088600003018651005ED8A003068751035ED880BD
:108870000001013602360301882F02D004D0000126
:1088800000011DEF44F00001030189BF03D0000186
:108890004FEF44F0011E021E012AD8B4022A000143
:1088A000DEEF45F0B40E0301746F756B5A0E766FF0
:1088B000776B0E0E786F010E796F7A6B7B6BFF0E04
:1088C000706F716B6F6B000103016F510308D8B0BB
:1088D00003D00001C0EF44F00001036A03016F51AF
:1088E0006925E96E6A510320EA6EEF52D8A403D0DD
:1088F0000001BBEF44F000010301712B703D02D079
:1089000004D0000100018AEF44F000016FC370F34E
:10891000BBEF44F0D89003016F35036A6725E96E19
:1089200068510320EA6EECCF7FF3ED52EFCF7EF378
:10893000D8907035036A6725E96E68510320EA6EA6
:10894000ECCF03F0ED52EF50016E7F51035CD8B0D5
:1089500003D00001BBEF44F00001D8A4B9EF44F00C
:10896000015003017E5DD8A003D00001BBEF44F0AD
:1089700000016FC370F303016F2B000164EF44F03B
:108980000301703D02D004D000010001CFEF44F09C
:108990000001FF0E016EFF0E026EF3EF45F0D8905E
:1089A00003017035036A740FE96E030E0320EA6E4B
:1089B000ECCF7FF3ED52EFCF7EF36B517E5D006E17
:1089C0006C517F59036E0050FF0A010F006E000EBC
:1089D00003560050726F03C073F373AF03D00001EE
:1089E0000DEF45F073510008D8A003D000010DEF42
:1089F00045F00001FF0AD8A407EF45F003017251CA
:108A00006708D8A003D000010DEF45F00001680E03
:108A10000301725F010E735B0001030173AF03D0AA
:108A2000000116EF45F000011CEF45F0680E030150
:108A30007227010E73230001D89003017035036A79
:108A40006725E96E68510320EA6EECCF03F0ED5222
:108A5000EF50916F03C092F3000179EC2BF000C04E
:108A60007EF301C07FF302C080F303C081F381C3B2
:108A700094F380C393F37FC392F37EC391F3800E8C
:108A80000301986F960E976F180E966F950E956F5F
:108A900000019BEC2BF000C082F301C083F302C005
:108AA00084F303C085F36EC392F36DC391F379EC45
:108AB0002BF085C38DF384C38CF383C38BF382C304
:108AC0008AF303C091F302C090F301C08FF300C09A
:108AD0008EF32AEC2DF000C086F301C087F302C0AC
:108AE00088F303C089F389C38DF388C38CF387C3EC
:108AF0008BF386C38AF30301916B906B200E8F6F0B
:108B0000820E8E6F00012AEC2DF003C08DF302C09F
:108B10008CF301C08BF300C08AF3FEEC2CF002C092
:108B20008BF301C08AF30B0E03018A257C6F000EC4
:108B30008B217D6F71510108D8A003D00001E8EFAF
:108B400045F0000173C303F003017251F2CF7EF3CD
:108B5000F29E03C0F7FF0001CCEC02F003017EBFE0
:108B6000F28E016E806B01C07FF3640E7F5D006E3C
:108B7000000E8059036E0050816F03C082F3196AA2
:108B8000F2BE198EF29EF46B0C0EF36F82C3F6F3F5
:108B900081C3F5F3000119EC09F019BEF28E02C091
:108BA00083F301C082F383C385F382C384F303019B
:108BB000876B640E866F0001EBEF43F002C003F099
:108BC000015003017C2703507D230001EEEF45F0A7
:108BD0000B0E03017C27000E7D23000103017C5155
:108BE000016E7D51026E00014CEF49F003017E6B76
:108BF000010E7F6F000103017F517C5DD8B003D06F
:108C000000010FEF46F00001D89003017E35010905
:108C10007E6F000103017F2B0001FBEF45F0030194
:108C20007B517E157D6F7D51016E0001000CFE0EA3
:108C300003017D6F7B517D15006ED89000307C6FF5
:108C40007C51016E0001000C03016C51E96E6D5105
:108C5000EA6E6EC3EFFF010E6C25E96E000E6D210A
:108C6000EA6E6FC3EFFF020E6C25E96E000E6D21F8
:108C7000EA6E70C3EFFF030E6C25016E000E6D21CE
:108C8000036E0150776F03C078F371C37BF3030E5B
:108C90007C6F0001F6EC45F078C3EAFF77C3E9FF8B
:108CA00001C0EFFF030E03016C25016E000E6D2164
:108CB000036E0150776F03C078F3030E6C25E96EE5
:108CC000000E6D21EA6EEF387A6FF00E7A1772C3DC
:108CD0007BF3040E7C6F0001F6EC45F003017A5142
:108CE00001107B6F78C3EAFF77C3E9FF7BC3EFFF17
:108CF000030E6C25016E000E6D21036E0150776F1F
:108D000003C078F3030E6C25E96E000E6D21EA6E48
:108D1000D890EF347A6F78C3EAFF77C3E9FF7AC35C
:108D2000EFFF040E6C25016E000E6D21036E0150E5
:108D3000776F03C078F373C37BF3000117EC46F041
:108D400078C3EAFF77C3E9FF01C0EFFF040E030118
:108D50006C25016E000E6D21036E0150776F03C00C
:108D600078F3040E6C25E96E000E6D21EA6ED89042
:108D7000EF347A6F78C3EAFF77C3E9FF7AC3EFFF76
:108D80007653D8A403D00001D4EF46F00001040EBE
:108D900003016C25016E000E6D21036E0150E96E1A
:108DA00003C0EAFFEF800001050E03016C25016E90
:108DB000000E6D21036E0150776F03C078F374C30A
:108DC0007BF3010E7C6F0001F6EC45F078C3EAFFFF
:108DD00077C3E9FF01C0EFFF050E03016C25016EAB
:108DE000000E6D21036E0150776F03C078F3050EFE
:108DF0006C25E96E000E6D21EA6E7A6BEFB07A8F0A
:108E000075C37BF3000117EC46F003017A510110A2
:108E10007B6F78C3EAFF77C3E9FF7BC3EFFF0001F5
:108E200076EF49F06AC303F003016951E96E03C0AC
:108E3000EAFF6B51EF5C706F000ED8807055716F58
:108E4000010ED8A0E806726F010E715D006E000E73
:108E50007259036E00506E5DD8A403D0000137EF45
:108E600047F0D8A003D0000187EF47F000010301CD
:108E70006F6B000103016E516F5DD8A003D000013C
:108E80006AEF47F000016AC303F003016951E96E1C
:108E900003C0EAFFEF506F25036A6725016E685132
:108EA00003220150726F03C073F3036A6F516C2584
:108EB000E96E6D510320EA6EEF50746F73C3EAFFE1
:108EC00072C3E9FF74C3EFFF000103016F2B0001C0
:108ED0003AEF47F06AC303F003016951716F03C0B1
:108EE00072F36AC303F06951E96E03C0EAFF6E5181
:108EF000EF24746F72C3EAFF71C3E9FF74C3EFFF1D
:108F0000010E016E00018BEF47F08BEF47F0000E72
:108F1000016E8BEF47F08AEF49F003015D6B4D0E58
:108F2000656F666B0A0E676F00014CEC3EF0030143
:108F30005D6B000103015D510308D8B003D000014F
:108F4000F2EF48F00001010E0301676F000108EC29
:108F500035F003015D510208D8B403D00001BCEF25
:108F600047F00001FF0E0301576FFF0E566F556B60
:108F7000546B0001D1EF48F0010E03015D25676FCE
:108F8000140E686FEA0E696F67C36AF3000103018C
:108F90006A2D02D004D000010001D4EF47F0000197
:108FA000090EC26E09EF48F003016A510208D8B4F5
:108FB00003D00001E1EF47F000010D0EC26E09EF92
:108FC00048F003016A510308D8B403D00001F8EF58
:108FD00047F00001FF0E0301576FFF0E566F556BF0
:108FE000546B000E016E0001CFEF48F009EF48F01E
:108FF00003016A510408D8B403D0000105EF48F01A
:109000000001110EC26E09EF48F0FF0E016ECFEFA6
:1090100048F08150070B816E8A96170E006E002E65
:10902000FED7B00E03016825716F556B546B685104
:10903000CF5CD8B003D0000123EF48F00001FF0E51
:10904000016ECFEF48F003016851CF5CD8B003D078
:10905000000123EF48F00001C282CE50CFCF03F0D1
:1090600003016D6F03C06EF3000103017151CF5C0A
:10907000D8A003D0000192EF48F00001030169512C
:10908000CF5CD8B003D000014BEF48F00001FE0EDA
:10909000016ECFEF48F06EC370F36DC36FF3C2B2D1
:1090A0004FEF48F0C282CE50CFCF03F003016D6F77
:1090B00003C06EF3196AF2BE198EF29EF46BC4CF30
:1090C000F3F3010EF66FF56B000119EC09F019BE10
:1090D000F28E02C073F301C072F3C3500301722514
:1090E0006B6F000E73216C6F55516C5DD8B003D05F
:1090F000000190EF48F00001D8A488EF48F0030188
:109100006B51545DD8A003D0000190EF48F00001EE
:109110006CC355F36BC354F370C357F36FC356F36B
:1091200035EF48F0C290196AF2BE198EF29E030123
:10913000F46B68C3F3F3010EF66FF56B000119ECE5
:1091400009F019BEF28E02C003F001500301565F10
:109150000350575BE20E565F040E575BDC0E565F02
:10916000000E575B5751A808D8A003D00001CDEFDF
:1091700048F00001FF0AD8A4C7EF48F00301565198
:10918000EC08D8A003D00001CDEF48F00001FF0E9D
:109190000301576FFF0E566F0001000E016E01C0F4
:1091A0005EF3D89003015D35036A480FE96E030E44
:1091B0000320EA6E57C3ECFFED5256C3EFFFD89081
:1091C0005D35036A380FE96E030E0320EA6E55C35E
:1091D000ECFFED5254C3EFFF000103015D2B0001D2
:1091E0009AEF47F052EC3EF0010E0301676F000169
:1091F0004CEC3EF0030E0301686F400E676F020EE9
:109200006A6FE60E696F030E6C6F380E6B6F0001AC
:1092100055EF3EF001C05EF3030E0301686F480E88
:10922000676F030E6A6F400E696F020E6C6FF60E69
:109230006B6F030E6E6F500E6D6F0001EBEF3EF023
:1092400001C05EF3030E0301686F400E676F030EEB
:109250006A6F500E696F030E6C6F5A0E6B6F030EC0
:109260006E6F5C0E6D6F00013CEF40F001C05EF36D
:10927000030E0301686F480E676F030E6A6F500E8E
:10928000696F5BC36CF35AC36BF3E5C26EF3E4C260
:109290006DF3000152EF44F002C059F301C058F3DE
:1092A000E3EC3CF001C067F359C368F358C369F3BA
:1092B0005BC36AF35AC36BF3030E03016D6F5F0E5A
:1092C0006C6FDFC16EF337C36FF367C370F35CC3BA
:1092D00071F368C372F369C373F36AC374F36BC346
:1092E00075F366C376F3000124EF46F0010E030127
:1092F000686FE20E676F010E6A6FE10E696FE0C181
:109300006BF3030E6D6F5F0E6C6F060E6E6F0001D8
:1093100012EF47F00152D8A491EF49F0640E020118
:10932000FF6F0001CDEF4EF000EC16F00152D8B403
:109330009EEF49F0000E016EB4EF49F01EAAA5EFB2
:1093400049F0000E016EB4EF49F0400E016E010EBF
:10935000EA6E410EE96EEE6A012EABEF49F00101B3
:10936000816B926B010E016E00018DEF4AF04CC3D0
:1093700003F003014B514D6F03C04EF3196AF2BE67
:10938000198EF29E000198EC27F019BEF28E4EC3A2
:10939000EAFF4DC3E9FF01C0EFFF4AC303F0030139
:1093A00049514D6F03C04EF3196AF2BE198EF29EF9
:1093B0000001A0EC27F019BEF28E4EC3EAFF4DC3A8
:1093C000E9FF01C0EFFF4AC303F003014951E96E11
:1093D00003C0EAFF2A51EF5CD8A003D00001F5EFEB
:1093E00049F000010301292B00014AC303F00301E6
:1093F0004951E96E03C0EAFFEF502A6F48C303F0FA
:109400004751E96E03C0EAFF29C3EFFF0001E5EF12
:109410004AF0400ED88001018155016E0001000C18
:109420004BC303F003014A51E96E03C0EAFFEF505A
:10943000495D506F4E51505DD8B003D0000172EFBE
:109440004AF0000103014F6B000103014E514F5DD3
:10945000D8A003D0000155EF4AF00001036A0301D0
:109460004F514C25016E4D5103220150516F03C0E5
:1094700052F34BC303F04A51E96E03C0EAFFEF50C9
:109480004F25036A4725E96E48510320EA6EEF50E5
:10949000546F52C3EAFF51C3E9FF54C3EFFF000109
:1094A00003014F2B000125EF4AF04BC303F00301EA
:1094B0004A51516F03C052F34BC303F04A51E96E56
:1094C00003C0EAFF4E51EF24546F52C3EAFF51C369
:1094D000E9FF54C3EFFF010E016E000176EF4AF081
:1094E00076EF4AF0000E016E76EF4AF0CDEF4BF0CA
:1094F00003013C91196AF2BE198EF29E000104EC40
:1095000022F019BEF28E0152D8B48BEF4AF0000E51
:10951000016E32EF4CF094EF49F0010E0301676FDA
:10952000000108EC35F00301396B3A6B2DC33BF3B6
:10953000376B000103013CA103D000012DEF4CF07B
:10954000000103013A5139252D5DD8A403D0000153
:109550002DEF4CF0D8B003D000012DEF4CF00001FE
:1095600003013B07750E476F660E486F00018BECD9
:1095700038F03BC348F3CBEC38F003012B51395D95
:10958000D8A003D000019AEF4BF00001030139533A
:10959000D8B403D00001FEEF4AF000010201FEB58D
:1095A00003D00001FEEF4AF00001030E0301486FF3
:1095B000440E476F030E4A6F450E496F030E4C6F02
:1095C000460E4B6F0001B7EF49F0D30E0301476F12
:1095D000370E486F00018BEC38F044C348F3CBECF6
:1095E00038F045C348F3CBEC38F046C348F3CBEC36
:1095F00038F00201FE95000195EF4BF0010193BB9D
:1096000003D000014AEF4BF0000152C04AF32DC3D2
:109610004BF319EC3CF00101DF5101240301496FC8
:1096200049C34AF30A0E4B6F000119EC3CF000529B
:10963000D8A44AEF4BF009EC4AF001503408D8B0F6
:109640004AEF4BF0AC0E0301476F450E486F000127
:109650008BEC38F003013D6B000103013D513208F2
:10966000D8B003D000014AEF4BF00001036A0301B8
:109670003D51AC0FE96E010E0320EA6EEFCF47F3C8
:1096800047C348F30001CBEC38F003013D2B000148
:109690002DEF4BF009EC4AF001500308D8B095EFDC
:1096A0004BF0CB0E0301476F810E486F00018BEC2E
:1096B00038F009EC4AF0D890013003013725386FB3
:1096C0003851285DD8A003D000016AEF4BF00001AB
:1096D00028C338F303013851375DD8A003D0000107
:1096E00095EF4BF00001036A03013751E96E030E59
:1096F0000324EA6EEFCF47F347C348F30001CBECF6
:1097000038F0036A03013751140FE96E030E03208A
:10971000EA6EEFCF47F347C348F30001CBEC38F0D4
:109720000301372B00016AEF4BF00301392B0001D5
:10973000FAEF4BF003012C513A5DD8A003D00001A1
:10974000FAEF4BF0000109EC4AF001500208D8B0E2
:10975000F7EF4BF0CA0E0301476FEA0E486F0001A6
:109760008BEC38F009EC4AF001500508D8B0F7EF5F
:109770004BF0010E0301486FE20E476FE1C149F360
:10978000010E4B6FE00E4A6F030E4D6F3E0E4C6F95
:10979000060E4E6F000110EF4AF00152D8B4F3EFFD
:1097A0004BF003013D6B000103013D510508D8B0AA
:1097B00003D00001F1EF4BF00001036A03013D51BA
:1097C0003E0FE96E030E0320EA6EEFCF47F347C367
:1097D00048F30001CBEC38F003013D2B0001D4EF3E
:1097E0004BF0F5EF4BF0F7EF4BF0B2EF4BF003011E
:1097F0003A2B0001010E0301476F0001FDEC38F028
:10980000010E0301676F000108EC35F05EEC3AF0E1
:109810000152D8B418EF4CF0196AF2BE198EF29EBC
:109820007AEC21F019BEF28E0152D8A42BEF4CF045
:1098300003013C813A53D8B403D0000127EF4CF028
:109840000001140E0201FF6F00012BEF4CF0150E0A
:109850000201FF6F00019AEF4AF0000E03013CA1E4
:10986000010E016E000120EF4FF08150070BF0094F
:1098700003013B6F8150070B10093C6F8150070BB0
:109880003D6F3DC381FF070E93163A51CF5CD8B0B0
:1098900003D0000151EF4CF00001FF0E016EA5EF67
:1098A0004CF003013A51CF5CD8B003D0000151EF26
:1098B0004CF000013BC381FF140E006E002EFED75A
:1098C0003CC381FF130E006E002EFED700D03BC3B9
:1098D00081FF140E006E002EFED73CC381FF130ED5
:1098E000006E002EFED700D03BC381FF140E006E29
:1098F000002EFED73CC381FF130E006E002EFED754
:1099000000D03BC381FF140E006E002EFED73CC377
:1099100081FF130E006E002EFED700D03BC381FFE7
:10992000140E006E002EFED73CC381FF130E006E96
:10993000002EFED700D0010E0301456F00011CEC84
:1099400034F03DC381FF000E016ECEEF4CF0140EDB
:109950000301386F450E396F0A0E676F00014CEC3A
:109960003EF00301376B0001030137510308D8B003
:1099700003D00001D3EF4CF00001010E0301676F2B
:10998000000108EC35F0382CC8EF4CF0CAEF4CF071
:10999000D3EF4CF038C33AF335EF4CF00301372BDB
:1099A0000001B4EF4CF0010E0301676F00014CECB5
:1099B0003EF03DEF4FF0196AF2BE198EF29E1BEC9D
:1099C00016F019BEF28E196AF2BE198EF29E2FECB5
:1099D00010F019BEF28E0201FE93196AF2BE198EC2
:1099E000F29E0301AE6B0001C3EC10F019BEF28EC3
:1099F0000201FE91FF6B0301286B0101E06BE16B3B
:109A0000196AF2BE198EF29E0001B6EC1CF019BE66
:109A1000F28E0201FEA703D000011DEF4DF0000100
:109A2000EAEF3BF00152D8A41AEF4DF0010E02010B
:109A3000FF6F00010201FE8700013DEC3CF0010ECA
:109A40000301336F900E326FFF0E316F3481349308
:109A50003495356B00010201FEA103D0000147EFF0
:109A60004FF00001030134A303D0000141EF4DF09A
:109A70000001010E0301676F000108EC35F044EFAF
:109A80004DF003013493000103013251D8B4330780
:109A90003207313D02D004D00001000153EF4DF0F8
:109AA000000156EF4DF00301310700012EEC35F0B7
:109AB0000152D8B467EF4EF0C60E0301436F580E43
:109AC000446F00017DEC35F00152D8B485EF4DF0C4
:109AD000196AF2BE198EF29E0301EA6BD50EE96F88
:109AE000060EEB6F0001A3EC0FF019BEF28E0152CF
:109AF000D8B485EF4DF072EC2FF0010E0301676FC3
:109B0000000108EC35F07DEF4DF0C60E0301436F08
:109B1000B70E446F00017DEC35F00152D8B49FEFD1
:109B20004DF0080E0301386F2D0E376F3A6B500E53
:109B3000396F0001CFEC2DF00201FE850001CB0E44
:109B40000301436F850E446F00017DEC35F0015237
:109B5000D8B4FDEF4DF0CB0E0301456F850E466F77
:109B6000000133EC35F001503308D8A4FDEF4DF07F
:109B7000CB0E0301436F850E446F000193EC35F06B
:109B800002C039F301C038F303013851E96E39518D
:109B9000EA6E0101DF51EF5CD8B403D00001FDEFA4
:109BA0004DF00001CB0E0301436F850E446F0001A1
:109BB00093EC35F002C038F301C037F3010EEA6EC2
:109BC000AC0EE96E38C3E2FF37C3E1FF330E016E1E
:109BD000E6CFEEFF012EE8EF4DF00101938B00017F
:109BE000ACEF3CF0040E0301386F160E376F3A6B82
:109BF000500E396F0001CFEC2DF0750E0301436F4D
:109C0000660E446F00017DEC35F00152D8B462EF6E
:109C10004EF0750E0301456F660E466F000133EC82
:109C200035F0012C43EF4EF00301356B313D02D08E
:109C300004D00001000134EF4EF000011FC130F3E9
:109C4000750E0301436F660E446F000193EC35F00F
:109C500002C003F00150E96E03C0EAFFEF500301B8
:109C6000316F000141EF4EF00301305101011F5DE2
:109C7000D8A403D0000141EF4EF000010301348568
:109C8000000148EF4EF00301352BFF0E316F00014C
:109C9000E3EC3CF001C037F330C33EF337C33FF38E
:109CA00006EC3DF0CB0E0301436F810E446F0001C3
:109CB0007DEC35F00152D8B460EF4EF07CEF3DF012
:109CC00065EF4EF00301352B00016AEF4EF0030102
:109CD000352B0001C1EF3DF0030134A103D0000199
:109CE00082EF4EF0000103012853D8A403D00001F5
:109CF00082EF4EF000010201FEA303D000018BEFC2
:109D00004EF00001030135516408D8A003D00001D2
:109D100099EF4EF00001196AF2BE198EF29EFF0E05
:109D20000301AE6F0001C3EC10F019BEF28EB3EF69
:109D30004EF003012853D8A403D00001B3EF4EF036
:109D400000010201FEA303D00001B3EF4EF00001B9
:109D5000196AF2BE198EF29E0301AE6B0001C3ECCC
:109D600010F019BEF28E3DEC3CF003013153D8B433
:109D700003D00001F4EF4EF00001030134B503D02D
:109D80000001C9EF4EF00001030134950001F0EF2E
:109D90004EF030C337F38DEF47F0030134B103D0F9
:109DA0000001DAEF4EF000010301336B326B00016A
:109DB000EEEF4EF0040E0301325F000E335B33AF63
:109DC00003D00001E7EF4EF00001EEEF4EF0320E4F
:109DD0000201FF6F0301336B326B000152EC3EF066
:109DE000FF0E0301316F0001030133AF03D0000107
:109DF000FDEF4EF0000101EF4FF0280E0201FF6F62
:109E00000001030135516408D8A003D000010EEF12
:109E10004FF000010301336B326B00010301325339
:109E2000D8B403D0000145EF4FF0000103013353D4
:109E3000D8B403D0000145EF4FF0000178EF4AF0AD
:109E40000152D8B427EF4FF0000E28EF4FF0010E6B
:109E5000016E01B031EF4FF003013493000134EF94
:109E60004FF0030134830001030134A303D0000148
:109E700045EF4FF00001A7EF4CF0030134912FC3E1
:109E800033F32EC332F3356B00012BEF4DF0DBEFD4
:109E90004CF09EEF50F0F86AD09E0D8EEA6AE96AA7
:109EA0008A82C150C00B0F09C16E070EB46E01014A
:109EB000AA6BAB6B939B939D938F000131EF2BF0BB
:109EC0004EEF2BF00101938B080E0301386F2D0E1E
:109ED000376F3A6B500E396F0001CFEC2DF0AFEFBA
:109EE0002EF0AEEF32F0196AF2BE198EF29E030127
:109EF000AE6B0001C3EC10F019BEF28EC00EF21270
:109F00002BC1DFF1750E0301436F660E446F000134
:109F1000BFEC2EF0C60E0301436FB70E446F000175
:109F2000BFEC2EF00301306B010E316F000196EF94
:109F300033F0196AF2BE198EF29E020E0301AE6F63
:109F400000018DEC18F019BEF28E196AF2BE198E5E
:109F5000F29E2FEC10F019BEF28E0201FE97010165
:109F6000939F800E0201E36FE26B010193BF03D068
:109F700000017FEF50F000017FEF34F002C0E3F208
:109F800001C0E2F20201E56BE46BE3AF03D0000134
:109F9000CDEF4FF00001D3EF4FF0FF0E016E7DEFDC
:109FA00050F0D7EF4FF0E3C231F3E2C230F30301D8
:109FB0003153D8B403D00001EEEF4FF0000103019C
:109FC00030510908D8B003D00001EEEF4FF0000186
:109FD000FE0E016E7DEF50F003EF50F003013153A0
:109FE000D8B403D00001FFEF4FF00001030130515E
:109FF0006408D8A003D0000103EF50F00001FD0E6B
:10A00000016E7DEF50F00301326B0001030132510C
:10A010005A08D8B003D000017DEF50F00001196A52
:10A02000F2BE198EF29E0301F46B32C3F3F3F66BAA
:10A03000040EF56F000119EC09F019BEF28E02C092
:10A0400034F301C033F334C303F003013351F2CFCF
:10A0500035F3F29E03C0F7FF000108EC02F009009F
:10A06000F5CF03F0030135BFF28E305DD8B403D0D5
:10A07000000178EF50F0000103500301315DD8B4C6
:10A0800003D0000178EF50F00001196AF2BE198E7A
:10A09000F29E0301F46B32C3F3F3F66B040EF56F1B
:10A0A000000119EC09F019BEF28E02C034F301C0B0
:10A0B00033F3020E03013325016E000E3421036ECB
:10A0C0000150F2CF35F3F29E03C0F7FF000108EC18
:10A0D00002F00900F5CF03F0030135BFF28E020153
:10A0E000E46F03C0E5F2000E016E00017DEF50F059
:10A0F0000301322B000106EF50F088EF50F002010F
:10A10000E36B2A0EE26F860EE56FA00EE46F00018E
:10A110001BEF38F0196AF2BE198EF29EB6EC1CF0F5
:10A1200019BEF28E38EF39F0196AF2BE198EF29E1E
:0EA130002FEC10F019BEF28EDBEF4CF00300A6
:020000040001F9
:10F000008B94000CE553D8A409EFF8F0C76A230EDF
:10F01000C66EE52D10EFF8F0300EC66E800EC76E8E
:10F0200019EFF8F0949A94889496E4C0E5F002EF12
:10F03000F8F01FEFF8F0010EE46F12EFF8F08C9685
:10F04000000CC9CFEEF0ECC0C9FFC7A025EFF8F067
:10F05000C9CFEDF0ED51016E000C8C86000C1BEC5D
:10F06000F8F0570EEC6F21ECF8F0EC6B21ECF8F0B7
:10F0700001C0E3F02DECF8F0E3AF45EFF8F0010E3E
:10F08000016E49EFF8F049EFF8F0000E016E49EF1C
:10F09000F8F0000C006A016A026A036AF36BF46B11
:10F0A000F56BF66BF251F111F011EF11D8B48EEF50
:10F0B000F8F0200EF76FD890EB37EC37ED37EE37DE
:10F0C000F337F437F537F637F251F65DD8A475EF1C
:10F0D000F8F0F151F55DD8A475EFF8F0F051F45D5A
:10F0E000D8A475EFF8F0EF51F35DD8A087EFF8F0F2
:10F0F000EF51F35FF051D8A0F03DF45FF151D8A08B
:10F10000F13DF55FF251D8A0F23DF65FD8800036B0
:10F11000013602360336F72F5BEFF8F00000EA6A9B
:10F12000F30EE96E000CD851DC5DD8A0FCEFF8F0CE
:10F13000D8A4B0EFF8F0D751DB5DD8A0FCEFF8F021
:10F14000D8A4B0EFF8F0D651DA5DD8A0FCEFF8F013
:10F15000D8A4B0EFF8F0D951D55DD8B0FCEFF8F0F5
:10F16000D8C0EEF0D7C0EDF0D6C0ECF0D5C0EBF0D3
:10F17000F26BF16B010EF06F080EEF6F4AECF8F0D6
:10F18000EFCFDDF0ECCFDEF0ECCFDFF0ECCFE0F056
:10F19000D551D95D006ED651DA59016ED751DB5980
:10F1A000026ED851DC59036E0050DD25E16F01502D
:10F1B000DE21E26F0250DF21E36F0350E021E46FB4
:10F1C000E453D8A4F6EFF8F0E353D8A4F6EFF8F040
:10F1D000E2510008D8B0FAEFF8F0FF0AD8A4F6EF31
:10F1E000F8F0E1510708D8B0FAEFF8F0000E016E20
:10F1F00048EFF9F046EFF9F0DCC0EEF0DBC0EDF0DF
:10F20000DAC0ECF0D9C0EBF0F26BF16B010EF06FED
:10F21000080EEF6F4AECF8F0EFCFDDF0ECCFDEF048
:10F22000ECCFDFF0ECCFE0F0D951D55D006EDA51D4
:10F23000D659016EDB51D759026EDC51D859036E95
:10F240000050DD25E16F0150DE21E26F0250DF2129
:10F25000E36F0350E021E46FE453D8A442EFF9F0E8
:10F26000E353D8A442EFF9F0E2510008D8B046EFDA
:10F27000F9F0FF0AD8A442EFF9F0E1510708D8B03D
:10F2800046EFF9F0000E016E48EFF9F0010E016E45
:10F2900063EFFAF0DCC0EEF0DBC0EDF0DAC0ECF0CA
:10F2A000D9C0EBF0F26BF16B010EF06F080EEF6F4F
:10F2B0004AECF8F0EFCF00F0ECCF01F0ECCF02F029
:10F2C000ECCF03F00150026E0050016E000CF76BA2
:10F2D000F86B010EF96FDA6AD96AFC6BEF0EFB6FFF
:10F2E000EA6AF30EE96EFCC0E2FFFBC0E1FFF9C081
:10F2F000FAF0D890E550EE02F350F723F450F823DB
:10F30000FA2F7AEFF9F0F7C0DEFFF8C0F7F0F86BEC
:10F31000D8B0F82BFB2BF92BF9510508D8A470EFC6
:10F32000F9F0BDEFF9F0E6C0EEF0E5C0EDF0E4C0B5
:10F33000ECF0E3C0EBF0F26BF16B010EF06F080E36
:10F34000EF6F4AECF8F001C0E8F000C0E7F0EE6BB8
:10F35000ED6BE8C0ECF0E7C0EBF0EEC0F2F0EDC012
:10F36000F1F0ECC0F0F0EBC0EFF0F66BF56B010ED6
:10F37000F46F080EF36F67EFF9F00050E35D006E75
:10F380000150E459016E0250E559026E0350E659EE
:10F39000036E01C0EAF000C0E9F0D890E737E83723
:10F3A000EAA1D4EFF9F0E781036AE80EE96E03C041
:10F3B000EAFFEFCFEBF0EBC0ECF021ECF8F0036AE2
:10F3C000E70EE96E03C0EAFFEFCFEBF0EBC0ECF025
:10F3D00021ECF8F0036AE90EE96E03C0EAFFEFCF13
:10F3E000EBF0EBC0ECF021ECF8F0000C2FECF8F0B7
:10F3F0000152D8A400EFFAF0000E016E46EFFAF0C9
:10F400001BECF8F0680EEC6F21ECF8F0DCC0E6F0D5
:10F41000DBC0E5F0DAC0E4F0D9C0E3F093ECF9F03A
:10F42000EC6B21ECF8F0EC6B21ECF8F0EC6B21ECE0
:10F43000F8F0EC6B21ECF8F0E26BE16BE251E05D8F
:10F44000D8A042EFFAF0D8A42BEFFAF0DF51E15D3B
:10F45000D8B042EFFAF0DEC003F0DD51E36F03C035
:10F46000E4F0EC6B21ECF8F0E4C0EAFFE3C0E9FF64
:10F4700001C0EFFFDD2BD8B4DE2BE12BD8B4E22B9B
:10F480001EEFFAF02DECF8F0010E016E000C2FECDF
:10F49000F8F00152D8A451EFFAF0000E016E31EFEE
:10F4A000FCF0C8C0D8F0C7C0D7F0C6C0D6F0C5C001
:10F4B000D5F008C0DCF007C0DBF006C0DAF005C00C
:10F4C000D9F093EFF8F00152D8B4FEEFFAF0C8C0CB
:10F4D000DCF0C7C0DBF0C6C0DAF0C5C0D9F04AEC3A
:10F4E000F9F002C0CEF001C0CDF0CCC0D2F0CBC05C
:10F4F000D1F01BECF8F00A2C8FEFFAF0540EEC6F01
:10F5000021ECF8F0C8C0E6F0C7C0E5F0C6C0E4F0F2
:10F51000C5C0E3F093ECF9F0EC6B21ECF8F00A5085
:10F520000208D8A4A5EFFAF0560EEC6F21ECF8F023
:10F53000C8C0E6F0C7C0E5F0C6C0E4F0C5C0E3F05F
:10F5400093ECF9F0EC6B21ECF8F0CB51CC11D8B482
:10F55000CFEFFAF0CD510808D8A4B4EFFAF0CE2DD1
:10F56000B4EFFAF0CFEFFAF0CAC003F0C951D56F8B
:10F5700003C0D6F0EC6B21ECF8F0D6C0EAFFD5C0A2
:10F58000E9FF01C0EFFFC92BD8B4CA2BCD2BD8B4EB
:10F59000CE2BCB51D8B4CC07CB07A5EFFAF02DEC8E
:10F5A000F8F0CB51CC11D8B4FAEFFAF0CB51D15DD1
:10F5B000006ECC51D259036E0050C525D56F035053
:10F5C000C621D66F000EC721D76F000EC821D86F95
:10F5D000D8C0DCF0D7C0DBF0D6C0DAF0D5C0D9F0A7
:10F5E000CAC0DEF0C9C0DDF0CCC0E0F0CBC0DFF0B7
:10F5F000F6ECF9F0010E016E31EFFCF0C851085C39
:10F60000D8A01DEFFCF0D8A41BEFFBF0C751075C9E
:10F61000D8A01DEFFCF0D8A41BEFFBF0C651065C90
:10F62000D8A01DEFFCF0D8A41BEFFBF0C551055C82
:10F63000D8A01DEFFCF0CB51C525D56FCC51C6210C
:10F64000D66F000EC721D76F000EC821D86F0850A3
:10F65000D85DD8A01DEFFCF0D8A444EFFBF0075014
:10F66000D75DD8A01DEFFCF0D8A444EFFBF0065006
:10F67000D65DD8A01DEFFCF0D8A444EFFBF00550F8
:10F68000D55DD8A01DEFFCF0CCC0D2F0CBC0D1F03E
:10F69000C551055CD56FC6510658D66FC75107587E
:10F6A000D76FC8510858D86F08C0DCF007C0DBF02E
:10F6B00006C0DAF005C0D9F04AECF9F00150D55D8A
:10F6C000D36F0250D659D46FCE6BCD6BC8C0DCF06F
:10F6D000C7C0DBF0C6C0DAF0C5C0D9F0CAC0DEF0E2
:10F6E000C9C0DDF0D4C0E0F0D3C0DFF0F6ECF9F033
:10F6F000D351CB5FD451CC5BD351C927D451CA234A
:10F700001BECF8F00A2CA2EFFBF0540EEC6F21EC8E
:10F71000F8F0D351C525D56FD451C621D66F000E50
:10F72000C721D76F000EC821D86FD8C0E6F0D7C068
:10F73000E5F0D6C0E4F0D5C0E3F093ECF9F0EC6B63
:10F7400021ECF8F00A500208D8A4C4EFFBF0560EE2
:10F75000EC6F21ECF8F0D351C525D56FD451C621FB
:10F76000D66F000EC721D76F000EC821D86FD8C042
:10F77000E6F0D7C0E5F0D6C0E4F0D5C0E3F093ECF6
:10F78000F9F0EC6B21ECF8F0CB51CC11D8B4EEEFE2
:10F79000FBF0CD510808D8A4D3EFFBF0CE2DD3EF6A
:10F7A000FBF0EEEFFBF0CAC003F0C951D56F03C008
:10F7B000D6F0EC6B21ECF8F0D6C0EAFFD5C0E9FF3B
:10F7C00001C0EFFFC92BD8B4CA2BCD2BD8B4CE2B98
:10F7D000CB51D8B4CC07CB07C4EFFBF02DECF8F03D
:10F7E000CB51CC11D8B419EFFCF0CB51D15D006EE8
:10F7F000CC51D259036E0050C525D56F0350C62198
:10F80000D66F000EC721D76F000EC821D86FD8C0A1
:10F81000DCF0D7C0DBF0D6C0DAF0D5C0D9F0CAC072
:10F82000DEF0C9C0DDF0CCC0E0F0CBC0DFF0F6EC1C
:10F83000F9F0010E016E31EFFCF0C8C0DCF0C7C07A
:10F84000DBF0C6C0DAF0C5C0D9F0CAC0DEF0C9C06E
:10F85000DDF0CCC0E0F0CBC0DFF0F6ECF9F0010E4B
:10F86000016E000CF250036EF29EA69CA68EA6843A
:10F870000F01550EA76EAA0EA76EA68200000350B8
:10F88000F2120001000C979C8E9C000C2FECF8F0FB
:10F890000152D8A450EFFCF0000E016E6CEFFCF0AA
:10F8A0001BECF8F0680EEC6F21ECF8F0C8C0E6F045
:10F8B000C7C0E5F0C6C0E4F0C5C0E3F093ECF9F0D2
:10F8C000EC6B21ECF8F0EC6B21ECF8F0EC6B21EC3C
:10F8D000F8F0EC6B21ECF8F089EFFDF0979C8E8C42
:10F8E0009DEFFDF08B849FEFFDF0C46BC351C45DB1
:10F8F000D8B091EFFCF0C451C125016E000EC221B9
:10F90000036E0150C56F03C0C6F0EC6B21ECF8F03C
:10F91000C6C0EAFFC5C0E9FF01C0EFFFC42B76EF08
:10F92000FCF0ACEFFDF0C4C003F0C351E96E03C0BE
:10F93000EAFFEF50C76FC6C003F0C551E96E03C0C0
:10F94000EAFFEF50C86FC8C0C9F0C7C0C8F0C9C04F
:10F95000C7F0C251C81BC839006E0F0E0016005008
:10F96000C81BC839006EF00E00160050C71BC83106
:10F97000006E003200321F0E00160050C71BC8393F
:10F98000006EF00E00160050D89000360050C81BD4
:10F99000C4C003F0C351E96E03C0EAFFC7C0EFFF64
:10F9A000C6C003F0C551E96E03C0EAFFC8C0EFFF4F
:10F9B000000CF86AD09EEA6AE96A0F0EC16E070E63
:10F9C000B46E8A8200ECF8F0C06BBF6BBC6B050EA6
:10F9D000BB6FBA6B400EB96FC86BC76BC66BC56B9C
:10F9E000CA6BA50EC96FCC6B0A0ECB6F47ECFAF051
:10F9F000A5C00DF0A6C00EF0036AC00EE96E03C0EC
:10FA0000EAFFA7C0EFFF036ABF0EE96E03C0EAFF7B
:10FA1000A8C0EFFFA9C00BF0B66BB56B106A116AF6
:10FA20000C6A0B500C5CD8B02DEFFEF0C46BC36BAE
:10FA3000BCC0C2F0BBC0C1F0C4C0C8F0C3C0C7F0F6
:10FA4000C2C0C6F0C1C0C5F0CA6BA50EC96FCC6BF1
:10FA5000040ECB6F47ECFAF0036AB00EE96E03C0F8
:10FA6000EAFFA5C0EFFF036AAF0EE96E03C0EAFF2D
:10FA7000A6C0EFFF036AB80EE96E03C0EAFFA7C095
:10FA8000EFFF036AB70EE96E03C0EAFFA8C0EFFFFD
:10FA9000AF51C00BB16FB051B26FAF513F0BB36FED
:10FAA000B051000BB46FB551B15DD8A45DEFFDF05E
:10FAB000B651B25DD8B46FEFFDF0B353D8A465EF83
:10FAC000FDF0B453D8B46FEFFDF0D08CF86AB2C03B
:10FAD000F7FFB1C0F6FFA68832ECFCF0F86AB2C0BE
:10FAE000B6F0B1C0B5F0040EBB27000EBC2343EC4A
:10FAF000FCF0C46BC36BBAC0C2F0B9C0C1F0C4C0E3
:10FB0000C8F0C3C0C7F0C2C0C6F0C1C0C5F046EF60
:10FB1000FCF0BE6BBD6BBE51B85DD8A028EFFEF007
:10FB2000D8A498EFFDF0B751BD5DD8B028EFFEF036
:10FB3000BDA9A1EFFDF06EEFFCF072EFFCF0A5EFB8
:10FB4000FDF043ECFCF000ECF8F0C26B150EC16F59
:10FB5000100EC36F75EFFCF0100EB927000EBA231C
:10FB6000D08CF86AB0C0F7FFAFC0F6FFF650070BB5
:10FB7000006EF80EF6160A00EA6A150EE96E100E0F
:10FB8000026E02C001F00050022602040709026E54
:10FB9000022AF6500066D7EFFDF0010F3F0BD8A404
:10FBA000D7EFFDF0A688090032ECFCF00A000066F1
:10FBB000E4EFFDF0EECFF5FF0152D8B4E5EFFDF034
:10FBC0000F000106E7EFFDF000060B000C00070E2A
:10FBD000F614070AD8A4EFEFFDF032ECFCF0022E89
:10FBE000C9EFFDF0F86AF86AB0C0F7FFAFC0F6FFE2
:10FBF000EA6A150EE96E100E006E0900F5CFEEFFF1
:10FC0000002EFDEFFDF0F86A136A13500F08D8A01C
:10FC10001FEFFEF0150E1324E96EEA6AD8B0EA2A47
:10FC2000EFCFC1F0C1C0C2F0C46B100EC36FC66B82
:10FC3000110EC56F93ECFCF0132A05EFFEF0100EC9
:10FC4000AF27000EB023BD2BD8B4BE2B8BEFFDF039
:10FC50002DECF8F00C2A11EFFDF00DC0C2F0C46BD2
:10FC6000100EC36FC66B110EC56F93ECFCF00EC087
:10FC7000C2F0C46B100EC36FC66B110EC56F93EC50
:10FC8000FCF0BA6B400EB96FBC6B050EBB6F105227
:10FC9000D8B44FEFFEF01152D8A40CEFFDF000ECF9
:10FCA000F8F043ECFCF0FF000300FFFFFFFFFFFF55
:020000040030CA
:0E00000000220C0E83018100FFC0FFE0FF40D4
:00000001FF
